:100000000C9485000C94A2000C94A2000C94A20005
:100010000C94A4000C94A2000C94A2000C94A200D6
:100020000C94A2000C94A2000C94A2000C94A200C8
:100030000C94A2000C94A2000C94A2000C94A200B8
:100040000C94A2000C94A2000C94A2000C94A200A8
:100050000C94A200942F122E622E8A2E912E942E92
:100060009A2EC62E122F362F7F2F842F912FF12DEF
:10007000C12F1030173025302C3034303C30433015
:100080004A304D30533056305D3066306B308B30F7
:1000900084309130712E4A30682E983005A84CCDAE
:1000A000B2D44EB93836A9020C50B9918688083CB2
:1000B000A6AAAA2ABE000000803F0664EC1B3C04EE
:1000C000BC163E3BE5B93CC93C37C29E5A3D66046E
:1000D00098083EEA69AAAA3E000000803F0706058C
:1000E000040302010010203040506070717273747C
:1000F0007576776757473727170403122130405129
:100100006273746556473726150011241FBECFE56C
:10011000D8E0DEBFCDBF11E0A0E6B0E0E6E4FEE649
:1001200002C005900D92A633B107D9F711E0A6E3FE
:10013000B1E001C01D92A23CB107E1F70E94EE02BE
:100140000C9421370C9400001F920F920FB60F925F
:1001500011242F933F938F939F93EF93FF9315BA9F
:10016000C39A20E030E0E091C101F0E083E0EE0FBF
:10017000FF1F8A95E1F7E20FF31FE358FE4F8081DE
:100180008BBB98B3822F8F5F8770987F892B88BB3A
:100190002F5F3F4F2830310531F7C3982091C101BF
:1001A00081E090E002C0880F991F2A95E2F785BB95
:1001B0008091C1018F5F8093C1018091C10188301E
:1001C00011F41092C101FF91EF919F918F913F9196
:1001D0002F910F900FBE0F901F9018959FEF9ABB15
:1001E0008FEE87BB94BB8FE181BB1BBA15BA80E150
:1001F00088BB80E682BB8AE083BD85B5856085BD0E
:1002000085B5886085BD14BC89B7806889BF10BC7E
:1002100089E189B986E880BD88E18AB91CB808956A
:100220001F9340E050E020E030E014E004C040E0E4
:1002300050E020E030E082B3812782BB5F9BFECF9D
:100240008CB190E08F3F910531F45F9BFECF8CB174
:1002500090E0009761F3FA0193E0EE0FFF1F9A958B
:10026000E1F7E20FF31FE35CFE4F80832730310597
:1002700049F44730510519F40E948A0DD8CF4F5FD9
:100280005F4FD7CF2F5F3F4FD6CFCF93DF93C09134
:100290007200D0917300939A2196CE010E947B3612
:1002A00088EE93E00E94B50B9398929A859B1AC0B2
:1002B000B49B1BC0869B1CC0809172009091730000
:1002C00088539F4FC817D90780F488EE93E00E94A7
:1002D000B50B9298939A859B05C0B49B06C08699EE
:1002E000DBCF06C022E030E005C021E030E002C0F4
:1002F00023E030E0C901DF91CF9108951F9382B3CD
:100300001092C0011092BF0110E1A4C010923C01F4
:1003100010923B018FC082B3812782BB1092BE0135
:100320001092BD0113C06091BF017091C001809116
:100330003B0190913C010E94DB058091BD019091B1
:10034000BE0101969093BE018093BD014091BD0115
:100350005091BE014830510534F31092390110928A
:100360003801E0917000F0917100DF01AA0FBB1F0E
:100370006091720070917300409136015091370185
:1003800020E030E024C06F5F7F4FB49B16C1859999
:1003900009C07093730060937200509337014093CB
:1003A0003601A6C0869B03C080E090E00AC070932F
:1003B0007300609372005093370140933601ACC0D4
:1003C0000196AC018E179F07DCF32F5F3F4F2A1772
:1003D0003B07CCF270937300609372005093370127
:1003E0004093360130933901209338011092BE01B9
:1003F0001092BD010FC06091BF017091C0010E94B9
:100400008E058091BD019091BE0101969093BE0131
:100410008093BD014091BD015091BE0180913B018F
:1004200090913C014830510534F3019690933C0182
:1004300080933B0180913B0190913C0108970CF423
:100440006ACF8091BF019091C00101969093C00145
:100450008093BF018091BF019091C00108970CF477
:1004600055CF1092BE011092BD0110E19DC01092B7
:10047000C0011092BF0188C082B3812782BB109255
:100480003C0110923B016EC04091BD015091BE01F4
:100490000E94DB05109239011092380180917000A2
:1004A0009091710064E070E00E94FE35AB01E09134
:1004B0007200F0917300609136017091370120E075
:1004C00030E038C03196B49909C0F0937300E093DE
:1004D0007200709337016093360177C085990FC021
:1004E000F0937300E09372007093370160933601CC
:1004F000309339012093380122E030E06CC0869BB4
:1005000003C080E090E010C0F0937300E0937200AD
:10051000709337016093360130933901209338018D
:1005200023E030E058C00196BC0184179507DCF346
:100530002F5F3F4F241735072CF2F0937300E093A1
:100540007200709337016093360130933901209324
:10055000380180913B0190913C01019690933C01C0
:1005600080933B0180913B0190913C016091BF01E0
:100570007091C001883091050CF486CF6F5F7F4F7A
:100580007093C0016093BF018091BF019091C00141
:1005900008970CF471CF8091BD019091BE01019636
:1005A0009093BE018093BD018091BD019091BE01E9
:1005B00008970CF45CCF94980FC07093730060930D
:1005C00072005093370140933601309339012093E4
:1005D000380121E030E0C9011F9108957F928F9288
:1005E0009F92AF92BF92CF92DF92EF92FF920F93C2
:1005F0001F93DF93CF93CDB7DEB7C15CD0400FB66A
:10060000F894DEBF0FBECDBF0E94EE0078940E942A
:100610007E0181E08093C1010E94450183309105F4
:1006200009F02DC280E00E94DF0880E690E00E9481
:10063000FA1812BA969A80E00E94DF085E010894C8
:10064000A11CB11C54E0752E41E4C42ED12CCC0E5B
:10065000DD1E31E8832E912C8C0E9D1E80E00E94C1
:10066000DF0886E690E00E94FA1801E010E06FC013
:1006700010923C0110923B012FC01092C0011092C9
:10068000BF011BC00E94763669E070E00E94FE3513
:100690008C016091BF017091C00180913B019091EC
:1006A0003C01A8010E94940D8091BF019091C0016E
:1006B00001969093C0018093BF018091BF019091FA
:1006C000C0010897FCF280913B0190913C0101969A
:1006D00090933C0180933B0180913B0190913C01C0
:1006E00008975CF21092BE011092BD012AC084E608
:1006F00090E00E94B50B8AE76FEF7FEF0E94C40B7A
:1007000081E090E00AC0879B03C000E21EE402C0C3
:100710000F5F1F4F81E29EE4869B8C018EE40032C6
:1007200018078CF3879904C08EE401321807FCF295
:100730008091BD019091BE0101969093BE0180937E
:10074000BD018091BD019091BE0107975CF3869930
:100750008FCF80E00E94DF0888E690E00E94FA18C0
:100760009EC00E94763669E070E00E94FE35AC01C2
:1007700080E090E060E070E00E94B40D0E94763668
:1007800069E070E00E94FE35AC0180E090E064E03A
:1007900070E00E94B40D0E94763669E070E00E941D
:1007A000FE35AC0182E090E062E070E00E94B40DA2
:1007B0000E94763669E070E00E94FE35AC0182E06E
:1007C00090E066E070E00E94B40D0E94763669E029
:1007D00070E00E94FE35AC0184E090E060E070E0E3
:1007E0000E94B40D0E94763669E070E00E94FE35EA
:1007F000AC0184E090E064E070E00E94B40D0E94DF
:10080000763669E070E00E94FE35AC0186E090E04B
:1008100062E070E00E94B40D0E94763669E070E0FC
:100820000E94FE358C0186E090E066E070E0A80151
:100830000E94B40D1092BE011092BD012AC084E640
:1008400090E00E94B50B8AE76FEF7FEF0E94C40B28
:1008500081E090E00AC0879B03C000E21EE402C072
:100860000F5F1F4F81E29EE4869B8C018EE4003275
:1008700018078CF3879904C08EE401321807FCF244
:100880008091BD019091BE0101969093BE0180932D
:10089000BD018091BD019091BE0107975CF38699DF
:1008A00060CF80E00E94DF088AE690E00E94FA189C
:1008B00001E010E047C010923C0110923B011AC0C9
:1008C0000E94763669E070E00E94FE35BC0180939C
:1008D000BF017093C00180913B0190913C010E9447
:1008E000F30D80913B0190913C01019690933C0166
:1008F00080933B0180913B0190913C01089704F368
:100900001BC084E690E00E94B50B8AE76FEF7FEF93
:100910000E94C40B81E090E00AC0879B03C000E204
:100920001EE402C00F5F1F4F81E29EE4869B8C0194
:100930008EE4003218078CF3879904C08EE40132EC
:100940001807FCF28699B7CF80E00E94DF088CE69A
:1009500090E00E94FA185EC000E010E0F501E00FA0
:10096000F11F70820E947636F601E00FF11F68E0F9
:1009700070E00E94FE3580830F5F1F4F0034110529
:1009800069F700E010E0C501B6014AE70E94B5151D
:1009900086E990E00E94B50B0F5F1F4F08301105EC
:1009A00091F734C000E010E0C501B6014AE70E94AB
:1009B000B51586E990E00E94B50B0F5F1F4F083018
:1009C000110591F702C0869B02C0879BFCCFEE24E5
:1009D000FF240E9476368C010E9476369C01C80165
:1009E00060E470E00E94FE35F601E80FF91FC901CE
:1009F00068E070E00E94FE3580830894E11CF11CE1
:100A000080E2E816F10429F7869B02C0879BCACFD3
:100A1000869B02C08699A0CF80E00E94DF088EE608
:100A200090E00E94FA18C4010E94B73200E024C08E
:100A3000869B02C0879BFCCF0E94763666E070E002
:100A40000E94FE35182F282F30E0802F90E082275B
:100A5000932786709070892B39F4C901039666E05C
:100A600070E00E94FE35182FC401602F412F28EC42
:100A700030E00E946A23012F869BF0CDDBCF8230CD
:100A8000910531F480E00E94DF0894980E941001E3
:100A900001E010E0C8010E94D22D0F5F1F4F03320A
:100AA0001105B4F7F7CF089778F477FD0DC06830DB
:100AB000710554F457FD08C090E0483051050CF022
:100AC00091E081E0982701C090E0892F0895FF927E
:100AD0000F931F93CF93DF93F82E8B01EA010E94AF
:100AE00053058823A9F0FE0183E0EE0FFF1F8A95CE
:100AF000E1F7E00FF11FE35CFE4F208181E090E021
:100B000002C0880F991FFA94E2F7809582238083B0
:100B1000DF91CF911F910F91FF900895FF920F9356
:100B20001F93CF93DF93F82E8B01EA010E945305A8
:100B30008823A9F0FE0193E0EE0FFF1F9A95E1F7DD
:100B4000E00FF11FE358FE4F208181E090E002C0EA
:100B5000880F991FFA94E2F7809582238083DF91B2
:100B6000CF911F910F91FF900895FF920F931F93C4
:100B7000CF93DF93F82E8B01EA010E94530588235F
:100B8000A1F0FE0123E0EE0FFF1F2A95E1F7E00F31
:100B9000F11FE35CFE4F208181E090E002C0880FEE
:100BA000991FFA94E2F7282B2083DF91CF911F91B0
:100BB0000F91FF900895FF920F931F93CF93DF93B0
:100BC000F82E8B01EA010E9453058823A1F0FE0153
:100BD00033E0EE0FFF1F3A95E1F7E00FF11FE35806
:100BE000FE4F208181E090E002C0880F991FFA94A7
:100BF000E2F7282B2083DF91CF911F910F91FF9077
:100C000008952F923F924F925F926F927F928F92B0
:100C10009F92AF92BF92CF92DF92EF92FF920F938B
:100C20001F93DF93CF93CDB7DEB72C970FB6F89411
:100C3000DEBF0FBECDBF281B390B061B170BE41AF6
:100C4000F50A37FD05C0A1E0B0E0BA87A98704C066
:100C5000EFEFFFEFFA87E9873C872B8737FF05C067
:100C6000309521953F4F3C872B8717FD05C021E02C
:100C700030E038872F8304C0AFEFBFEFB887AF8372
:100C800017FF03C0109501951F4FF7FC05C0E1E069
:100C9000F0E0FE83ED8304C02FEF3FEF3E832D8312
:100CA000F7FE04C0F094E194F108F394AB85BC85A1
:100CB000AA0FBB1FBC83AB83F801EE0FFF1FFA83A3
:100CC000E9831701220C331C2B853C852017310743
:100CD0000CF444C02E153F05DCF17F01E21AF30A43
:100CE0008101021B130B3C014A015B014424552482
:100CF00028C0C301B501A4010E94DB051E141F0416
:100D000044F48F819885A80EB91EAB81BC81EA1A84
:100D1000FB0A1016110644F4ED81FE818E0E9F1E13
:100D20002B813C81021B130B89819A81E80EF91EED
:100D3000020D131D0894411C511CA985BA856A0E29
:100D40007B1E6301EB85FC854E165F0694F290C016
:100D50002B853C85021713070CF448C00E151F05A0
:100D60000CF444C0EB80FC80E01AF10AD101A01B16
:100D7000B10BBC87AB873B014A016C01442455246D
:100D800030C0C601B301A4010E94DB051E141F047C
:100D900044F4E985FA85CE0EDF1E29813A81E21AF4
:100DA000F30A8B859C851816190654F4AD81BE8113
:100DB0008A0E9B1EE981FA818E1B9F0B9C878B8775
:100DC0002B813C81E20EF31E8B859C85820D931D49
:100DD0009C878B870894411C511CAF81B8856A0E93
:100DE0007B1E53014016510664F242C009811A81EC
:100DF0000E191F09EB81FC81EE19FF09FC87EB87B7
:100E00003A015B016C01442455242EC0C601B50192
:100E1000A3010E94DB051016110634F42F813885DA
:100E2000A20EB31E021913098B859C85181619068C
:100E300044F4A985BA85CA0EDB1E821993099C87E2
:100E40008B87E981FA810E0F1F1F2B853C858B81D3
:100E50009C81280F391F3C872B870894411C511C0B
:100E6000AD81BE816A0E7B1E43014E145F0474F295
:100E7000C601B501A4010E94DB052C960FB6F894BB
:100E8000DEBF0FBECDBFCF91DF911F910F91FF90BD
:100E9000EF90DF90CF90BF90AF909F908F907F901A
:100EA0006F905F904F903F902F900895FF920F9317
:100EB0001F93CF93DF93F82E8B01EA010E94530515
:100EC000882389F033E0CC0FDD1F3A95E1F7C00F9E
:100ED000D11FC358DE4F888190E002C09595879559
:100EE000FA94E2F78170DF91CF911F910F91FF90FB
:100EF00008952130310519F40E94DB0508950E9400
:100F00008E050895FF920F931F93CF93DF93F82ED2
:100F10008B01EA010E9453058823A1F0FE0143E002
:100F2000EE0FFF1F4A95E1F7E00FF11FE358FE4F68
:100F3000208181E090E002C0880F991FFA94E2F7C7
:100F400028272083DF91CF911F910F91FF90089563
:100F5000CF93DF93FC01DA01E901681779071CF4EC
:100F6000CB01BF01FC01ED93FC9379836883DF9192
:100F7000CF9108958830910598F420E030E053E057
:100F8000880F991F5A95E1F74FEFFC01E20FF31F0D
:100F9000E358FE4F40832F5F3F4F28303105A9F7BC
:100FA00008958830910590F420E030E063E0880FE8
:100FB000991F6A95E1F7FC01E20FF31FE358FE4F1A
:100FC00010822F5F3F4F28303105A9F708959C010B
:100FD0008830910530F581E090E002C0880F991FBC
:100FE0002A95E2F7982F40E050E012C0FB01E20F93
:100FF000F31FE358FE4F8081892B80832F5F3F4F83
:101000002830310599F74F5F5F4F4830510549F05F
:1010100020E030E0BA01E3E0660F771FEA95E1F7E0
:10102000E5CF08959C018830910538F581E090E086
:1010300002C0880F991F2A95E2F7982F909540E0FB
:1010400050E012C0FB01E20FF31FE358FE4F808116
:10105000892380832F5F3F4F2830310599F74F5FF9
:101060005F4F4830510549F020E030E0BA01F3E02D
:10107000660F771FFA95E1F7E5CF0895883091055F
:1010800098F420E030E04FEFF901A3E0EE0FFF1FEE
:10109000AA95E1F7E80FF91FE358FE4F40832F5F51
:1010A0003F4F2830310581F708958830910590F43D
:1010B00020E030E0F901B3E0EE0FFF1FBA95E1F751
:1010C000E80FF91FE358FE4F10822F5F3F4F283083
:1010D000310581F70895893749F08A37F9F0883763
:1010E000A1F5862F90E00E94E707089570E0683030
:1010F000710558F520E030E08FEFF90193E0EE0F35
:10110000FF1F9A95E1F7E60FF71FE358FE4F808324
:101110002F5F3F4F2830310581F7089570E0683028
:10112000710598F420E030E083E0660F771F8A9520
:10113000E1F78FEFFB01E20FF31FE358FE4F8083CF
:101140002F5F3F4F28303105A9F70895893749F0BF
:101150008A37F1F0883791F5862F90E00E941208C7
:10116000089570E06830710548F520E030E0F9013D
:1011700053E0EE0FFF1F5A95E1F7E60FF71FE35814
:10118000FE4F10822F5F3F4F2830310581F70895C1
:1011900070E06830710590F420E030E043E0660FC5
:1011A000771F4A95E1F7FB01E20FF31FE358FE4F6B
:1011B00010822F5F3F4F28303105A9F7089540E096
:1011C00050E010C0FB01E20FF31FE358FE4F808395
:1011D0002F5F3F4F28303105A9F74F5F5F4F4830F1
:1011E000510549F020E030E0BA01E3E0660F771FD7
:1011F000EA95E1F7E7CF089540E050E010C0FB0129
:10120000E20FF31FE35CFE4F80832F5F3F4F2830D8
:101210003105A9F74F5F5F4F4830510549F020E095
:1012200030E0BA01F3E0660F771FFA95E1F7E7CFF8
:101230000895EF92FF920F931F93CF93DF93DC01FA
:10124000EB01F9012817390714F4D901FC010C1737
:101250001D071CF4CE01E8018C01E416F5061CF410
:10126000CA01A7017C0131968FEF90E09C0102C07A
:10127000220F331FEA95E2F7209502C0880F991FCD
:10128000AA95E2F728230EC0FB01EA0FFB1FE358E3
:10129000FE4F8081822B808311960A171B07A4F7CB
:1012A0004F5F5F4FE416F50644F0DE01BA0183E0BC
:1012B000660F771F8A95E1F7F0CFDF91CF911F91ED
:1012C0000F91FF90EF900895CF92DF92EF92FF92EF
:1012D0000F931F93CF93DF93DC01F9012817390790
:1012E00014F4D901FC01061717071CF4CB01B8014F
:1012F0008C01E416F5061CF4CA01A7017C0181E00B
:1013000090E09C010E2E02C0220F331F0A94E2F7D8
:101310000A2E02C0880F991F0A94E2F7C22EC82A2B
:1013200031968FEF90E09C0102C0220F331FEA95A7
:10133000E2F7D22ED09402C0880F991FAA95E2F747
:10134000D8229A0121C0A617B70749F0A017B10704
:1013500031F02417350719F02E153F0539F4FE0139
:10136000EA0FFB1FE358FE4FD08208C0FE01EA0FD0
:10137000FB1FE358FE4F80818C29808311960A174A
:101380001B070CF72F5F3F4FE216F30644F0DB011B
:10139000E90193E0CC0FDD1F9A95E1F7F0CFDF91E3
:1013A000CF911F910F91FF90EF90DF90CF90089514
:1013B0006F927F928F929F92AF92BF92CF92DF9265
:1013C000EF92FF920F931F93CF93DF933C014B015A
:1013D0005A0169012817390714F439016C010815FD
:1013E00019051CF4C40148018C01EA14FB041CF427
:1013F000C50157017C010894C11CD11C8FEF90E0FE
:101400009C010C2C02C0220F331F0A94E2F70894AF
:10141000C108D1082095062C02C0880F991F0A9494
:10142000E2F72823D50143E0AA0FBB1F4A95E1F755
:10143000FD01E80DF91DE358FE4F2083A00FB11FF9
:10144000A358BE4F2C93D70133E0AA0FBB1F3A9588
:10145000E1F7FD01E80DF91DE358FE4F2083A00FD1
:10146000B11FA358BE4F2C93E40115C0C301BE01A8
:10147000A5010E94DB05C301BE01A7010E94DB0597
:10148000C601BE01A5010E94DB05C601BE01A70180
:101490000E94DB0521960C171D0744F7E50115C0D6
:1014A000C301B401AE010E94DB05C301B801AE0166
:1014B0000E94DB05C601B401AE010E94DB05C60136
:1014C000B801AE010E94DB052196EC16FD0644F73B
:1014D000DF91CF911F910F91FF90EF90DF90CF9010
:1014E000BF90AF909F908F907F906F9008956F5FA7
:1014F0007F4F2FEF30E0A90102C0440F551F6A95BE
:10150000E2F7BA01609502C0220F331F8A95E2F715
:10151000862F82230895482F282F30E082958695C4
:101520008270942F991F9927991F892B942F969534
:10153000969596959470892B46954870842B220F2A
:10154000331F922F9071892B220F331F220F331FCD
:10155000922F9072892B220F331F220F331F922F4D
:101560009074892B220F331F220F331F822B089573
:101570002F923F924F925F926F927F928F929F92A3
:10158000AF92BF92CF92DF92EF92FF920F931F9391
:10159000DF93CF93CDB7DEB766970FB6F894DEBF73
:1015A0000FBECDBF2C015B014A011901670128174D
:1015B00039073CF412012901C8018B015C016A0161
:1015C00047013101641875080A151B0544F4B5017B
:1015D000601B710B882777FD8095982F07C00A192B
:1015E0001B09B801882777FD8095982F0E94F43356
:1015F0007B018C01B301882777FD8095982F0E948D
:10160000F4339B01AC01C801B7010E9459336D83CB
:101610007E838F839887310164187508C814D904B4
:1016200044F4B4016C197D09882777FD8095982FC3
:1016300007C0C818D908B601882777FD8095982F6C
:101640000E94F4337B018C01B301882777FD8095DC
:10165000982F0E94F4339B01AC01C801B7010E948E
:10166000593369837A838B839C83642CC501AA27B1
:1016700097FDA095BA2F8D879E87AF87B88BC40141
:10168000AA2797FDA095BA2F898B9A8BAB8BBC8B21
:101690004BC06D897E8964197509882777FD80950F
:1016A000982F0E94F4335B016C016D817E818F81E4
:1016B0009885A60195010E94E1347B018C016D851E
:1016C0007E858F8598890E94F4339B01AC01C80107
:1016D000B7010E94EE320E94C63369877A878B87F2
:1016E0009C8769817A818B819C81A60195010E94EA
:1016F000E1347B018C0169897A898B899C890E94FC
:10170000F4339B01AC01C801B7010E94EE320E9484
:10171000C6339B01AC018D899E89698570E0422F9B
:1017200050E00E94DB056394A62DB0E0BE8BAD8B2C
:101730002A163B060CF0ADCF66960FB6F894DEBFC6
:101740000FBECDBFCF91DF911F910F91FF90EF9012
:10175000DF90CF90BF90AF909F908F907F906F90D1
:101760005F904F903F902F9008950BC020E00000B5
:10177000000000000000000000002F5F2A35B9F7CC
:101780000197009799F708952F923F924F925F9299
:101790006F927F929F92AF92BF92CF92DF92EF9221
:1017A000FF920F931F93CF93DF93982E5B01CC246E
:1017B000DD24A7E02A2E312C8FEFA8168FEFB80674
:1017C00011F4760103C07101EC18FD0800E010E08F
:1017D000270108944108510837010894611C711CC5
:1017E0003AC08FEFA8168FEFB80611F4C30101C0FD
:1017F000C201AC018AE7981649F4C801BE010E94F3
:101800005607282FC801BE01A70119C089E79816FD
:1018100051F4C801BA01AE010E945607282FC80131
:10182000B701AE010CC088E7981661F4CA01BE0189
:10183000A8010E945607282FC701BE01A80130E069
:101840000E9479072196C830D10559F60F5F1F4FC6
:101850000830110519F0C0E0D0E0C3CF0894C11CD6
:10186000D11C88E0C816D10409F0A6CF8FEFA816C6
:101870008FEFB80619F0EE24FF2403C0F7E0EF2E37
:10188000F12C00E010E01FC08AE7981621F4C8018F
:10189000BE01A7010DC089E7981621F4C801B70160
:1018A000AE0106C088E7981629F4C701BE01A80159
:1018B0000E948E052196C830D10531F70F5F1F4F6A
:1018C0000830110519F0C0E0D0E0DECFDF91CF91F4
:1018D0001F910F91FF90EF90DF90CF90BF90AF904E
:1018E0009F907F906F905F904F903F902F900895C2
:1018F000DF93CF93CDB7DEB7C054D0400FB6F89486
:10190000DEBF0FBECDBFDE011196EDE7F1E080E452
:1019100001900D928150E1F740E050E0BE016F5F11
:101920007F4F18C08C91F90193E0EE0FFF1F9A953D
:10193000E1F7E40FF51FE358FE4F8083189621501E
:1019400030408FEF2F3F380769F74F5F5F4F4830C8
:10195000510531F0DB01A40FB51F27E030E0E2CFE5
:10196000C05CDF4F0FB6F894DEBF0FBECDBFCF9186
:10197000DF9108958F929F92AF92BF92CF92DF92A4
:10198000EF92FF920F931F93DF93CF93CDB7DEB704
:10199000C054D0400FB6F894DEBF0FBECDBFDE01FD
:1019A0001196EDE7F1E080E401900D928150E1F7AE
:1019B0000E94DF08EE24FF244E010894811C911C34
:1019C00017C0F60181916F010E948B0AF501E00FAB
:1019D000F11FE358FE4F80830F5F1F4F0830110542
:1019E00081F70894E11CF11CF8E0EF16F10469F0AE
:1019F000C70123E0880F991F2A95E1F76401C80EFB
:101A0000D91E00E010E05C01DCCFC05CDF4F0FB6F8
:101A1000F894DEBF0FBECDBFCF91DF911F910F9124
:101A2000FF90EF90DF90CF90BF90AF909F908F90FE
:101A300008958F929F92AF92BF92CF92DF92EF92D2
:101A4000FF920F931F93DF93CF93CDB7DEB7C054B0
:101A5000D0400FB6F894DEBF0FBECDBFDE011196A9
:101A6000EDE7F1E080E401900D928150E1F70E94F2
:101A7000DF08AA24BB244E010894811C911C2AC0B3
:101A8000F701808190E0002E02C0959587950A9419
:101A9000E2F780FF05C0C801B601A5010E94DB0581
:101AA0000F5F1F4F0830110559F70894E11CF11C16
:101AB0000894C108D108FFEFCF16FFEFDF0619F039
:101AC00000E010E0DDCF0894A11CB11C88E0A8164E
:101AD000B10461F0750143E0EE0CFF1C4A95E1F79B
:101AE000E80CF91C37E0C32ED12CEACFC05CDF4FE5
:101AF0000FB6F894DEBF0FBECDBFCF91DF911F911F
:101B00000F91FF90EF90DF90CF90BF90AF909F909C
:101B10008F900895ADE7B1E0EDE3F1E080E401904E
:101B20000D928150E1F70895CF92DF92EF92FF92EC
:101B30000F931F93CF93DF936C017B018A01C0E069
:101B4000D0E006C0C601B701AE010E94DB052196B8
:101B5000C017D107BCF3DF91CF911F910F91FF9078
:101B6000EF90DF90CF9008958F929F92AF92BF92A7
:101B7000CF92DF92EF92FF920F931F93CF93DF9359
:101B80007C018B014A01C0E0D0E05C010894A11CFB
:101B9000B11C6B010894C11CD11C15C0C701B80150
:101BA000AE010E94DB05C501B801AE010E94DB0554
:101BB000C701B601AE010E94DB05C501B601AE0149
:101BC0000E94DB052196C815D90544F3DF91CF911A
:101BD0001F910F91FF90EF90DF90CF90BF90AF904B
:101BE0009F908F900895CF92DF92EF92FF920F9384
:101BF0001F93CF93DF936C017B0100E010E00DC0D9
:101C0000C0E0D0E0CE01B601A8010E94DB0521961C
:101C1000C830D105B9F70F5F1F4F0E151F0584F3AC
:101C2000DF91CF911F910F91FF90EF90DF90CF90B8
:101C30000895CF93DF93EC01DC0120E030E014C085
:101C4000A830B10574F4283031055CF4FD0183E05F
:101C5000EE0FFF1F8A95E1F7E20FF31FE358FE4FE7
:101C600060832F5F3F4F1197C217D3074CF7CA010C
:101C70000E94B50BCE01DF91CF9108950F931F9372
:101C8000CF93DF938B01EA01892B51F080E190E043
:101C9000BE01A8010E94190E019797FFF9CF0AC053
:101CA00080E090E0BE01A8010E94190E01968031EB
:101CB0009105C4F3DF91CF911F910F9108957F9209
:101CC0008F929F92AF92BF92CF92DF92EF92FF924C
:101CD0000F931F93CF93DF93E82EF62E742E690196
:101CE000C0E0D0E027E0822E912C98E0A92EB12C04
:101CF00087E0781669F484010C1B1D0BA5014C1BB1
:101D00005D0B8E2D90E06F2D70E00E948E050AC055
:101D1000AE01415050408E2D90E06F2D70E00E943A
:101D20008E058E018E2D90E06F2D70E0A8010E942F
:101D3000DB05C6010E94B50B2196C830D105C1F65E
:101D4000DF91CF911F910F91FF90EF90DF90CF9097
:101D5000BF90AF909F908F907F900895CF92DF9229
:101D6000EF92FF920F931F93CF93DF936C017B0150
:101D70000894E108F1088B0102501040080F191F68
:101D800025C0C0E0D0E0F8018081682F70E06F705E
:101D9000707082958F7090E0AE010E945607282FD8
:101DA000F8018181682F70E06F70707082958F707C
:101DB00090E0AE0130E00E9479072196C830D1054D
:101DC00011F70894E108F108015010401E141F0497
:101DD000C4F2C0E0D0E0F6018081682F70E06F703F
:101DE000707082958F7090E0AE010E948E052196F2
:101DF000C830D10581F7DF91CF911F910F91FF90EE
:101E0000EF90DF90CF9008955F926F927F928F92C4
:101E10009F92AF92BF92CF92DF92EF92FF920F9379
:101E20001F93DF93CF93CDB7DEB76C970FB6F894BF
:101E3000DEBF0FBECDBF4C01562E3A0180E05E01E1
:101E40000894A11CB11CB5014CE150E00E94572D33
:101E5000CC24DD243FC0852D6F2D4E2D0E94712D89
:101E6000882341F080E090E067E070E0A8010E94E4
:101E7000DB0507C080E090E067E070E0A8010E9409
:101E80008E050F5F1F4FFA948FEFF81621F7C401EC
:101E90000E94B50BC5016CE170E00E94AE0EE394A8
:101EA00088E0E81629F000E010E037E0F32ED3CF09
:101EB00000E010E0C4010E94B50BC5016CE170E0C8
:101EC0000E94AE0E0F5F1F4F0431110599F7089461
:101ED000C11CD11CC614D70414F4EE24E4CF00E0D6
:101EE00010E07E010894E11CF11CC4010E94B50BB6
:101EF000C7016CE170E00E94AE0E0F5F1F4F0A3009
:101F0000110599F76C960FB6F894DEBF0FBECDBFE2
:101F1000CF91DF911F910F91FF90EF90DF90CF90C5
:101F2000BF90AF909F908F907F906F905F9008953B
:101F30002F923F924F925F926F927F928F929F92D9
:101F4000AF92BF92CF92DF92EF92FF920F931F93C7
:101F5000DF93CF93CDB7DEB7A1970FB6F894DEBF6E
:101F60000FBECDBF3C016B0156E0852E912C8C0E2F
:101F70009D1E80E0B4014CE150E00E94572D1E01EF
:101F80000894211C311C240143C0B1010E94AE2DD4
:101F90007101F701808100E010E0A82EBB2487E0EA
:101FA00090E0801B910B950102C0359527958A958D
:101FB000E2F720FF08C080E090E067E070E0A80151
:101FC0000E94DB0507C080E090E067E070E0A801B8
:101FD0000E948E050F5F1F4F0830110501F7C401E5
:101FE0006CE170E00E94AE0EC3010E94B50B089434
:101FF000E11CF11CE414F50461F60894C11CD11C29
:10200000C2016CE170E00E94AE0EC3010E94B50BEC
:10201000F6018081882309F0B8CF00E010E046E0A7
:10202000E42EF12CEC0EFD1EC7016CE170E00E9465
:10203000AE0EC3010E94B50B0F5F1F4F0C3111058F
:1020400099F7A1960FB6F894DEBF0FBECDBFCF9122
:10205000DF911F910F91FF90EF90DF90CF90BF9095
:10206000AF909F908F907F906F905F904F903F9038
:102070002F9008959F92AF92BF92CF92DF92EF92EE
:10208000FF920F931F93DF93CF93CDB7DEB7609787
:102090000FB6F894DEBF0FBECDBF5C016B0181E0CF
:1020A0008E010F5F1F4FB80140E150E00E94572D95
:1020B000EE24FF24902E012F15C0A7014770507009
:1020C00084E090E060E070E00E94DB05C6010E94C1
:1020D000B50B892D902F6CE170E00E94AE0E089434
:1020E000E11CF11CEA14FB0444F360960FB6F8946B
:1020F000DEBF0FBECDBFCF91DF911F910F91FF903B
:10210000EF90DF90CF90BF90AF909F9008957F9217
:102110008F929F92AF92BF92CF92DF92EF92FF92F7
:102120000F931F93DF93CF93CDB7DEB76C970FB6A6
:10213000F894DEBF0FBECDBF4C015B0180E08E0185
:102140000F5F1F4FB8014CE150E00E94572D74E023
:10215000E72EF12CCC24DD24702E012F2AC00E9402
:1021600076360894E108F10863E070E00E94FE35DD
:10217000E80EF91E88E0E816F10424F067E0E62E88
:10218000F12C04C0F7FE02C0EE24FF24872D902F0F
:102190006CE170E00E94AE0E80E090E067E070E0DD
:1021A000A7010E94DB05C5010E94B50B0894C11C64
:1021B000D11CC814D9049CF26C960FB6F894DEBFFB
:1021C0000FBECDBFCF91DF911F910F91FF90EF9088
:1021D000DF90CF90BF90AF909F908F907F900895A9
:1021E0002F923F924F925F926F927F928F929F9227
:1021F000AF92BF92CF92DF92EF92FF920F931F9315
:10220000DF93CF93CDB7DEB7EC970FB6F894DEBF70
:102210000FBECDBF9FA78EA769AB7AAB48ABDE01DF
:102220001196E4E7F0E080E201900D928150E1F731
:102230001DA61CA69E012F5F3F4F3CAF2BAFD4C104
:10224000222433248824992444245524C40101964B
:102250002114310451F44C018430910539F441E0EA
:10226000242E312C8824992401C04C01C40133E070
:10227000880F991F3A95E1F76BAC7CAC681A790A24
:10228000AA24BB24E7E0EFA32FE130E0620E731E27
:10229000E1E0F0E0EC0FFD1FE80FF91FFAAFE9AF46
:1022A00026C088A96FA1402F0E94712D882361F05C
:1022B0002114310411F4F70101C0F6016081C80155
:1022C00070E0A5010E94DB050F5F1F4F0894C10855
:1022D000D1080894E11CF11C0830110511F708948D
:1022E000A11CB11CFFA1F150FFA3FF3F31F063011E
:1022F000E9ACFAAC00E010E0D4CF89A99AA90E9419
:10230000B50B80E00E94DF080894411C511C27E0B7
:102310004216510409F09ACF1EA21DA2662477240A
:1023200022243324C3010196EDA1FEA1EF2B59F421
:102330003C018430910541F421E030E03EA32DA31F
:102340006624772401C03C01C30123E0880F991F54
:102350002A95E1F74BAC5CAC481A590A88249924B9
:1023600037E038A7EFE1F0E04E0E5F1E21E030E0ED
:102370002C0F3D1F280F391F38AF2FAB2CC04E2D0F
:10238000415088A968A50E94712D882369F08DA10C
:102390009EA1892B11F4F60101C0F501808190E026
:1023A000B801A4010E94DB050894E11CF11C015056
:1023B00010400894A108B1080894C11CD11CF9E090
:1023C000EF16F104E1F60894811C911C28A5215018
:1023D00028A72F3F49F05201CFA8D8AC01E0E02E4A
:1023E000F12C07E010E0CBCF89A99AA90E94B50B88
:1023F00080E00E94DF080894211C311C37E023167E
:10240000310409F08FCF1CA21BA2662477241BA6DF
:102410001AA6C3010196EBA1FCA1EF2B59F43C01D4
:102420008430910541F421E030E03CA32BA36624E5
:10243000772401C03C01C30113E0880F991F1A954E
:10244000E1F74BAC5CAC481A590AAA24BB24B7E0AC
:102450002B2EEFE1F0E04E0E5F1E21E030E02C0F5E
:102460003D1F280F391F3EAB2DAB2AC048010894F1
:102470008108910888A9622D432D0E94712D88231F
:1024800069F08BA19CA1892B11F4F70101C0F60121
:102490006081C40170E0A5010E94DB050F5F1F4F42
:1024A0003A940894C108D1080894E11CF11CFFEF8C
:1024B0003F16E1F60894A11CB11C2A942F1641F096
:1024C0006201EDA8FEA801E010E0A7E03A2ECECF11
:1024D00089A99AA90E94B50B80E00E94DF082AA56D
:1024E0003BA52F5F3F4F3BA72AA72730310509F0B7
:1024F00090CF1AA219A26624772422243324C30180
:102500000196E9A1FAA1EF2B59F43C018430910521
:1025100041F421E030E03AA329A36624772401C0E6
:102520003C01C301F3E0880F991FFA95E1F74BAC2A
:102530005CAC481A590A8824992437E039A7EFE19E
:10254000F0E04E0E5F1E21E030E02C0F3D1F280F03
:10255000391F3CAB2BAB2BC088A969A5402F0E942B
:10256000712D882369F089A19AA1892B11F4F601B4
:1025700001C0F501808190E0B801A4010E94DB0553
:102580000894E11CF11C015010400894A108B10806
:102590000894C11CD11CF9E0EF16F104E9F6089487
:1025A000811C911C29A5215029A72F3F49F05201D8
:1025B000CBA8DCA8E1E0EE2EF12C07E010E0CCCFB8
:1025C00089A99AA90E94B50B80E00E94DF080894AF
:1025D000211C311C37E02316310409F090CF8CA563
:1025E0009DA501969DA78CA7ECA5FDA52EA53FA5B1
:1025F000E217F3070CF424CEEC960FB6F894DEBF86
:102600000FBECDBFCF91DF911F910F91FF90EF9043
:10261000DF90CF90BF90AF909F908F907F906F9002
:102620005F904F903F902F9008956F927F928F927E
:102630009F92AF92BF92CF92DF92EF92FF920F9351
:102640001F93CF93DF933C014B015A01CC24DD242F
:102650002CC00E9476368C010E9476367C010E9446
:102660007636FC01C80168E070E00E94FE358C01FE
:10267000C70168E070E00E94FE359C01CF0168E070
:1026800070E00E94FE35AC01C801B9010E94DB0573
:1026900021968C169D06ECF6C5010E94B50B80E0D4
:1026A0000E94DF080894C11CD11CC614D7041CF476
:1026B000C0E0D0E0EECFDF91CF911F910F91FF905E
:1026C000EF90DF90CF90BF90AF909F908F907F90D2
:1026D0006F900895CF93DF93C1E0D0E085E090E064
:1026E000BE0148EC50E00E9415132196C431D1057B
:1026F000A9F785E090E0BE0148EC50E00E94151378
:102700002197B9F7DF91CF910895DF92EF92FF9271
:102710000F931F93CF93DF938C0180E00E94DF081B
:10272000C0E0D0E0DD24DA94780111C0F901E80FAF
:10273000F91FE358FE4FD082019688309105B1F71A
:10274000C7010E94B50B2196C830D10549F080E041
:1027500090E09E0173E0220F331F7A95E1F7E6CFF8
:10276000C801880F991F800F911F0E94B50BC0E010
:10277000D0E011C0F901E80FF91FE358FE4F1082B5
:10278000019688309105B1F7C7010E94B50B2196DB
:10279000C830D10549F080E090E09E0153E0220F5F
:1027A000331F5A95E1F7E6CFDF91CF911F910F913B
:1027B000FF90EF90DF9008954F925F926F927F921B
:1027C0009F92AF92BF92CF92DF92EF92FF920F93C0
:1027D0001F93CF93DF93982E162F072F3A0180E097
:1027E0000E94DF08212F302FC9016C01C0E0D0E02A
:1027F000E7E04E2E512C35C06114710431F0F50123
:102800008081A201481B510904C0F7018081482F33
:1028100050E0FAE79F1619F4CE01B8010DC089E720
:10282000981621F4CE01BA01A80106C098E79916BE
:1028300029F4CA01B801AE010E94DB050F5F1F4FEA
:102840000894A11CB11C0894E11CF11C083011056E
:1028500099F62196E8E0F0E0CE0EDF1EC830D105F3
:1028600029F05601760100E010E0C6CFDF91CF914C
:102870001F910F91FF90EF90DF90CF90BF90AF909E
:102880009F907F906F905F904F9008952F923F920E
:102890004F925F926F927F928F929F92AF92BF9270
:1028A000CF92DF92EF92FF920F931F93DF93CF931C
:1028B000CDB7DEB7C158D0400FB6F894DEBF0FBE1B
:1028C000CDBFCF57DF4F8883C158D0402B013A018D
:1028D0004901B1E4AB2EB12CAC0EBD1EF501A1E84F
:1028E000CA2ED12CCC0EDD1E1192EC15FD05E1F7A0
:1028F00000E010E01E010894211C311C81E08816C4
:102900009104C9F414C00E94763660E470E00E941D
:10291000FE35E1E4F0E0EC0FFD1FE80FF91F8081C8
:10292000882389F70F5F1F4F91E0908316C0003412
:1029300011054CF312C082E08816910471F4003442
:1029400011055CF4E1E4F0E0EC0FFD1FE00FF11F76
:1029500080818F5F80830F5F1F4FF501EE24FF247E
:102960009081892F8150863010F49F5F9083808101
:10297000873019F40894E11CF11C3196EC15FD0523
:1029800079F7D101F50180814114510419F097E0E4
:10299000981B892F8C9331961196EC15FD0599F7AC
:1029A000C3010E94B50BCF57DF4F8881C158D0407B
:1029B000B10140E050E00E94DC1382B394E089272B
:1029C00082BB80E4E816F10409F098CFCF57DF4FBF
:1029D0000FB6F894DEBF0FBECDBFCF91DF911F9130
:1029E0000F91FF90EF90DF90CF90BF90AF909F90AE
:1029F0008F907F906F905F904F903F902F900895B1
:102A00003F924F925F926F927F928F929F92AF927E
:102A1000BF92CF92DF92EF92FF920F931F93DF93BB
:102A2000CF93CDB7DEB7C058D0400FB6F894DEBF15
:102A30000FBECDBF382E2B014A01390100E010E056
:102A40006E010894C11CD11C81E4E82EF12CEC0E1F
:102A5000FD1EF601E00FF11F10820E947636F7018D
:102A6000E00FF11F68E070E00E94FE3580830F5F89
:102A70001F4F0034110569F7EE24FF245E0108940E
:102A8000A11CB11C11E4C12ED12CCC0EDD1E1CC02A
:102A9000D8019C918081981710F49F5F9C930F5FE1
:102AA0001F4F31960C151D0599F7832DB501A30114
:102AB0000E94DC13C2010E94B50B0894E11CF11CBA
:102AC000B8E0EB16F10419F08501F601E1CFF80149
:102AD00027E0CE018F579F4F2193E817F907E1F7C1
:102AE000C4010E94B50BEE24FF244E010894811C02
:102AF000911C1FC080819C91891710F48F5F808387
:102B00008081981710F48150808331961196E017D8
:102B1000F10781F7832DB401A3010E94DC13C201E8
:102B20000E94B50B0894E11CF11C88E0E816F10442
:102B300019F0F501D601DECFC058DF4F0FB6F8947B
:102B4000DEBF0FBECDBFCF91DF911F910F91FF90E0
:102B5000EF90DF90CF90BF90AF909F908F907F903D
:102B60006F905F904F903F900895AC01DC01FB01A6
:102B700020E030E09C918081981710F49F5F9C9337
:102B80009C918081891710F491509C932F5F3F4F47
:102B9000119631962034310569F78AE7BA0140E091
:102BA00050E00E94DC1308952F923F924F925F9263
:102BB0006F927F928F929F92AF92BF92CF92DF924D
:102BC000EF92FF920F931F93DF93CF93CDB7DEB7B2
:102BD000C058D0400FB6F894DEBF0FBECDBF2C0159
:102BE0007B0100E010E05E010894A11CB11C54E0E0
:102BF000952E41E4C42ED12CCC0EDD1EF501E00F44
:102C0000F11F90820E947636F601E00FF11F68E016
:102C100070E00E94FE3580830F5F1F4F0034110566
:102C200069F700E010E031E4A32EB12CAC0EBD1E1C
:102C30006E010894C11CD11C3701C601B5014AE7D9
:102C40000E94B515C3010E94B50B0F5F1F4F0830DE
:102C5000110599F75701AA0CBB1CAA0CBB1CCC246C
:102C6000DD2491E4892E912C8C0E9D1E1E0108946A
:102C7000211C311C32C000E010E0C101B4014AE760
:102C80000E94B515C3010E94B50B0F5F1F4F08309E
:102C9000110599F7C5010E94B50BEE24FF240E948F
:102CA00076368C010E9476369C01C80160E470E0A3
:102CB0000E94FE35F401E80FF91FC90168E070E0D9
:102CC0000E94FE3580830894E11CF11C80E2E81626
:102CD000F10429F70894C11CD11CC414D5045CF27A
:102CE000C058DF4F0FB6F894DEBF0FBECDBFCF91F7
:102CF000DF911F910F91FF90EF90DF90CF90BF90E9
:102D0000AF909F908F907F906F905F904F903F908B
:102D10002F9008958F929F92AF92BF92CF92DF92A1
:102D2000EF92FF920F931F93CF93DF934C018B0190
:102D30006130710511F480E001C08FEF0E94DF085F
:102D4000C0E0D0E00E94763668E070E00E94FE3578
:102D5000B82EA92E0E94763668E070E00E94FE35FB
:102D6000D82EC92E0E94763668E070E00E94FE35AB
:102D7000F82EE92E0115110559F48B2D9A2D6D2D84
:102D80007C2D4F2D5E2D0E9456078130D9F40DC049
:102D900001301105B9F48B2D9A2D6D2D7C2D4F2D01
:102DA0005E2D0E945607882369F48B2D9A2D6D2D78
:102DB0007C2D4F2D5E2D98010E947907C4010E9441
:102DC000B50B219681E0CF3FD8070CF4BBCFDF9144
:102DD000CF911F910F91FF90EF90DF90CF90BF9018
:102DE000AF909F908F9008956F927F928F929F9255
:102DF000AF92BF92DF92EF92FF920F931F93CF9308
:102E0000DF933C015B014A0180E00E94DF0800E0A3
:102E100010E01FC00E94763662E070E00E94FE352E
:102E2000AC0163E0440F551F6A95E1F7481B590B4D
:102E3000C801BE010E94DB052196C830D10551F7BB
:102E40000F5F1F4F0830110521F4DD24EE24FF240D
:102E500030C0C0E0D0E0DECF0E947636EC010E94A8
:102E6000763668E070E00E94FE35082F8E1501F17D
:102E7000CE0168E070E00E94FE35182F8D15C1F07C
:102E800090E0602F70E040E050E00E9456078823F9
:102E900021F0812F602F40E003C0812F602F47E099
:102EA00095010E945F0EC4010E94B50BD12EE02E49
:102EB000F3948F2D90E08615970574F2DF91CF91F2
:102EC0001F910F91FF90EF90DF90BF90AF909F9078
:102ED0008F907F906F900895EF92FF920F931F93C2
:102EE000CF93DF9380E00E94DF0800E010E07FEEE8
:102EF000E72E72E0F72E47C080E00E94DF08CE0187
:102F00000E94B50B8FEF0E94DF0884E690E00E94DC
:102F1000B50BCE0166EF7FEF0E94FE3588EE93E0A1
:102F20000E94FE356F507040C60FD71F1C161D063D
:102F30001CF388EE93E00E94B50BCEEED2E080E069
:102F40000E94DF08C7018C1B9D0B0E94B50B8FEF01
:102F50000E94DF0884E690E00E94B50BCE0166EF88
:102F60007FEF0E94FE3588EE93E00E94FE356F50A1
:102F70007040C60FD71F1C161D060CF30F5F1F4FA6
:102F80000230110519F0CEEED2E0B6CFDF91CF912D
:102F90001F910F91FF90EF9008952F923F924F92C3
:102FA0005F926F927F928F929F92AF92BF92CF92D9
:102FB000DF92EF92FF920F931F93DF93CF93CDB7E2
:102FC000DEB72E970FB6F894DEBF0FBECDBF9A8343
:102FD00089837C836B835E834D8338872F831A8735
:102FE00009874F5F5F4F21F4F7E02F2E312C02C08D
:102FF00022243324E9E06E2E712C89819A81681A8B
:10300000790A0E947636B3010E94FE356C010E9457
:103010007636B3010E94FE357C01442455247CC0E1
:103020000E9476368C010E9476369C01C80163E0CE
:1030300070E00E94FE3501978C0D9D1D9E878D8747
:10304000181619061CF48615970514F0DE86CD8631
:10305000C90163E070E00E94FE358C010150104010
:103060000E0D1F1D101611061CF4061517050CF089
:1030700087018B816D817E810E94C40B8D849E842B
:10308000AA24BB2431C0EB81FC81EA37F10521F48D
:10309000C401B601A10115C08B819C8189379105BE
:1030A00021F4C401B101A6010CC0EB81FC81E83719
:1030B000F10549F44D855E854E0D5F1DC1016B859F
:1030C0007C850E94DB050894E11CF11C0894C11C5E
:1030D000D11C89819A81E816F906ACF20894A11CEA
:1030E000B11C0894811C911CE981FA81AE16BF06BF
:1030F0004CF46801EE24FF24C501800F911F9C87CA
:103100008B87E7CF89859A850E94B50B0894411C6F
:10311000511CCD84DE847801EF81F8854E165F0660
:103120000CF47ECF2E960FB6F894DEBF0FBECDBF47
:10313000CF91DF911F910F91FF90EF90DF90CF9093
:10314000BF90AF909F908F907F906F905F904F90C7
:103150003F902F900895AF92BF92CF92DF92EF925F
:10316000FF920F931F93CF93DF935C01CC24DD2458
:1031700033C00E94763664E070E00E94FE35EC01B8
:10318000EE24FF241AC00E9476368C010E94763607
:103190009C01C80168E070E00E94FE35FC01C90195
:1031A00068E070E00E94FE35BC01CF0147E050E0CE
:1031B0000E94DB050894E11CF11CEC16FD061CF3D3
:1031C00088EE93E00E94B50B8AE76FEF7FEF0E94D5
:1031D000C40B0894C11CD11CCA14DB0454F2DF9147
:1031E000CF911F910F91FF90EF90DF90CF90BF9004
:1031F000AF9008954F925F926F927F928F929F92BD
:10320000AF92BF92CF92DF92EF92FF920F931F93F4
:10321000DF93CF9300D000D00F92CDB7DEB76C0113
:103220003E010894611C711CB0E84B2E512C4AC021
:10323000B3010E94AE2DEE24FF2426C09201002E81
:1032400002C0359527950A94E2F7F401808190E059
:1032500028233923232B61F087E090E0B501A801F2
:103260000E94DB0586E090E0B501A8010E94DB0525
:103270000F5F1F4F0830110509F70894E11CF11C7E
:10328000F5E0EF16F10459F000E010E043018E0C78
:103290009F1CA2E0AA2EB12CAE0CBF1CCFCF00E029
:1032A00010E088EE93E00E94B50B88E76FEF7FEFA8
:1032B0000E94C40B0F5F1F4F0630110591F7089451
:1032C000C11CD11CF6018081882309F0B1CF00E038
:1032D00010E088EE93E00E94B50B88E76FEF7FEF78
:1032E0000E94C40B0F5F1F4F0830110591F70F901C
:1032F0000F900F900F900F90CF91DF911F910F9132
:10330000FF90EF90DF90CF90BF90AF909F908F9005
:103310007F906F905F904F900895AF92BF92CF9241
:10332000DF92EF92FF920F931F93CF93DF935C0195
:103330006B01EE24FF244FC0C0E0D0E08AE76FEFBE
:103340007FEF0E94C40B80E090E0BE0147E050E0B8
:103350000E94DB05CE0167E070E047E050E00E948C
:10336000DB0507E010E00C1B1D0B87E090E0B801C7
:1033700047E050E00E94DB05C80160E070E047E0F4
:1033800050E00E94DB0580E090E0B80147E050E0AB
:103390000E94DB05C80167E070E047E050E00E9452
:1033A000DB0587E090E0BE0147E050E00E94DB05CE
:1033B000CE0160E070E047E050E00E94DB05C6010E
:1033C0000E94B50B2196C730D10509F0B7CF87E031
:1033D00090E0E80EF91EAE14BF040CF0ADCFDF9103
:1033E000CF911F910F91FF90EF90DF90CF90BF9002
:1033F000AF900895AF92BF92CF92DF92EF92FF927B
:103400000F931F93CF93DF935C016B01EE24FF2496
:1034100032C0C0E0D0E08AE76FEF7FEF0E94C40BBC
:1034200080E090E0BE0147E050E00E94DB05CE0165
:1034300067E070E047E050E00E94DB0507E010E045
:103440000C1B1D0B87E090E0B80147E050E00E94A4
:10345000DB05C80160E070E047E050E00E94DB055A
:10346000C6010E94B50B2196C730D105A1F687E0B1
:1034700090E0E80EF91EAE14BF045CF6DF91CF9128
:103480001F910F91FF90EF90DF90CF90BF90AF9082
:1034900008952F923F924F925F926F927F928F92F8
:1034A0009F92AF92BF92CF92DF92EF92FF920F93D3
:1034B0001F93DF93CF93CDB7DEB7E8970FB6F8949D
:1034C000DEBF0FBECDBF9AAB89AB7CAB6BAB222E00
:1034D00080E00E94DF080E94763668E070E00E947B
:1034E000FE357C013C010E94763668E070E00E9467
:1034F000FE358C012C010E94763668E070E00E9457
:10350000FE35382F292F6C01FE013196CE01C19670
:103510009EAB8DAB00831183E282F38234832583DB
:1035200036968DA99EA9E817F907A1F711E0E12EBB
:10353000F12CB1E08B2E912CA1E0AA2EB12CFE0132
:103540003B97F8AFEFAB4BC20E94763663E070E07A
:103550000E94FE35892B71F50E94763663E070E09B
:103560000E94FE35009759F40E94763663E070E0C1
:103570000E94FE357C010894E108F1081BC08130EF
:10358000910559F40E94763663E070E00E94FE35A2
:103590004C010894810891080DC08230910551F4C6
:1035A0000E94763663E070E00E94FE355C0108946C
:1035B000A108B108FFEFEF16FFEFFF0699F44114E1
:1035C000510481F40E94763663E070E00E94FE357B
:1035D000019719F0EE24FF2403C0F1E0EF2EF12C47
:1035E00011E001C010E08FEF88168FEF980699F474
:1035F0006114710481F40E94763663E070E00E94E9
:10360000FE35019719F08824992403C0E1E08E2E3D
:10361000912C01E001C000E09FEFA9169FEFB906D1
:10362000A1F4C114D10489F40E94763663E070E0FD
:103630000E94FE35019719F0AA24BB2403C071E053
:10364000A72EB12C3324339401C03324E1E0EE16CD
:10365000F10499F4F7E04F16510479F40E9476369C
:1036600063E070E00E94FE35019719F0EE24FF241C
:1036700003C0EE24EA94FE2C11E081E08816910448
:1036800099F497E06916710479F40E94763663E044
:1036900070E00E94FE35019719F08824992403C038
:1036A00088248A94982C01E0E1E0AE16B104A1F4DC
:1036B000F7E0CF16D10481F40E94763663E070E023
:1036C0000E94FE35019719F0AA24BB2403C0AA2446
:1036D000AA94BA2C33243394112351F18114910408
:1036E00091F487E06816710439F06114710441F0B7
:1036F0000E94763680FD04C088248A94982C03C0EA
:1037000061E0862E912CA114B10491F497E0C916C2
:10371000D10439F0C114D10441F00E94763680FD05
:1037200004C0AA24AA94BA2C03C051E0A52EB12C3F
:10373000002351F1E114F10491F4E7E04E16510435
:1037400039F04114510441F00E94763680FD04C0E6
:10375000EE24EA94FE2C03C041E0E42EF12CA114E7
:10376000B10491F4F3E0CF16D10439F0C114D104BF
:1037700041F00E94763680FD04C0AA24AA94BA2C97
:1037800003C031E0A32EB12C332061F181149104E8
:1037900091F487E06816710439F06114710441F006
:1037A0000E94763680FD04C088248A94982C03C039
:1037B00021E0822E912CE114F104A1F497E0491646
:1037C000510421F4EE24EA94FE2C29C04114510442
:1037D00021F491E0E92EF12C08C00E94763680FF9A
:1037E00004C151C041145104B1F46114710441F495
:1037F000C114D10451F1E7E0CE16D10461F425C023
:10380000F7E06F16710439F4C114D104F1F087E0C8
:10381000C816D104D1F097E04916510461F561143E
:10382000710441F4C114D10481F0E7E0CE16D10453
:1038300011F50BC0F7E06F167104E9F4C114D1045F
:1038400021F087E0C816D104B1F40E94763663E017
:1038500070E00E94FE35009719F4EE24FF240BC09F
:103860008130910519F48824992405C0823091058E
:1038700011F4AA24BB244114510441F49FEFE9162A
:103880009FEFF90619F481E0E82EF12C6114710420
:1038900041F4EFEF8E16EFEF9E0619F401E0802E53
:1038A000912CC114D10441F4FFEFAF16FFEFBF0616
:1038B00019F411E0A12EB12C87E04816510439F417
:1038C00091E0E916F10419F4EE24EA94FE2CE7E005
:1038D0006E16710439F4F1E08F16910419F48824FE
:1038E0008A94982C87E0C816D10439F491E0A9167F
:1038F000B10419F4AA24AA94BA2C4E0C5F1C680CCB
:10390000791CCA0CDB1CE1E02E1679F4C201B3016C
:10391000A6010E94DB058BA99CA90E94B50BC201E0
:10392000B301A6010E948E0555C0F2E02F1651F496
:10393000C201B301A6010E9482078BA99CA90E9423
:10394000B50B48C083E0281609F044C0FE01B596C7
:1039500080819181978386838281938191878087FB
:10396000848195819387828736978FA998ADE817D0
:10397000F90771F75A8249827C826B82DE82CD829E
:103980008E010F5F1F4FF801628173814481558161
:10399000808191810E94DB050A5F1F4F8DA99EA93E
:1039A0000817190781F78BA99CA90E94B50B8E01F6
:1039B0000F5F1F4FF80162817381448155818081BF
:1039C00091810E948E050A5F1F4F8DA99EA908173D
:1039D000190781F7E9A9FAA93197FAABE9AB89A9E7
:1039E0009AA9892B09F0B0CD04C0EE24EA94FE2CEC
:1039F0004DCFE8960FB6F894DEBF0FBECDBFCF9186
:103A0000DF911F910F91FF90EF90DF90CF90BF90CB
:103A1000AF909F908F907F906F905F904F903F906E
:103A20002F900895CF92DF92EF92FF920F931F9302
:103A3000CF93DF93F82E6B01EA0180E00E94DF084C
:103A40008F2D90E00E94BA0710E10E94763664E064
:103A500070E00E94FE35E82E0E94763664E070E049
:103A60000E94FE35082F8E2D90E0602F70E04F2DC4
:103A700050E00E945607882341F38E2D602F4F2D72
:103A800096010E945F0ECE010E94B50B1150E9F61F
:103A9000DF91CF911F910F91FF90EF90DF90CF902A
:103AA00008958F929F92AF92BF92CF92DF92EF9242
:103AB000FF920F931F93CF93DF935C016B0180E024
:103AC0000E94DF08C0E0D0E003E0802E912C1C149F
:103AD0001D0414F0CE0103C0C4018C1B9D0BAC016E
:103AE0004C5F5F4F7401E81AF90ACA01BA019701E5
:103AF00087010E94D809C5010E94B50B80E00E9491
:103B0000DF082196C430D10511F7DF91CF911F91C5
:103B10000F91FF90EF90DF90CF90BF90AF909F906C
:103B20008F9008952F923F924F925F926F927F9263
:103B30008F929F92AF92BF92CF92DF92EF92FF92BD
:103B40000F931F93DF93CF9300D0CDB7DEB79A8347
:103B500089834B011A012901AA24BB242EEF622E6E
:103B60002FEF722E660E771E4BC0CC24DD2488E02A
:103B7000C816D10434F497E0E92EF12CEC18FD08B6
:103B800006C088EFE82E8FEFF82EEC0CFD1C80E0CD
:103B90000E94DF0881E090E00E94B50BF89480E07D
:103BA00090E060E070E040E050E0970187010E9403
:103BB000D8091214130414F40E94780C91E08916A9
:103BC000910421F0E3E08E16910411F40E94190D86
:103BD000F2E06F16710410F40E94BA0C7894C201DE
:103BE0000E94B50B80E00E94DF080894C11CD11C24
:103BF00080E1C816D10409F0BACF0894A11CB11C09
:103C0000E981FA81AE16BF060CF4AFCF0F900F908A
:103C1000CF91DF911F910F91FF90EF90DF90CF90A8
:103C2000BF90AF909F908F907F906F905F904F90DC
:103C30003F902F900895EF92FF920F931F93E82EDD
:103C4000F62E072F10E08E2D612F0E946B088F2D0E
:103C5000902F0E94B50B1F5F1830A9F717E080E086
:103C60000E94DF088E2D612F0E946B088F2D902FF0
:103C70000E94B50B115098F71F910F91FF90EF9094
:103C80000895EF92FF920F931F93E82EF62E072FC1
:103C900010E080E00E94DF088E2D612F0E946B08EB
:103CA0008F2D902F0E94B50B1F5F183091F717E0F2
:103CB00080E00E94DF088E2D612F0E946B088F2DFF
:103CC000902F0E94B50B115098F71F910F91FF9004
:103CD000EF900895AF92BF92CF92DF92EF92FF9252
:103CE0000F931F93CF93DF93C0E0D0E0BE0133E08A
:103CF000759567953A95E1F7882777FD8095982F18
:103D00000E94F4337B018C010E9444359B01AC017D
:103D10000E94EE3220E030E040E650E40E94EE32B5
:103D20000E94C1335B016C01C801B7010E94563388
:103D30009B01AC010E94EE3220E030E040E650E40E
:103D40000E94EE320E94C1337B018C01C501B70194
:103D500041E050E00E94DB05C501B70141E050E0C1
:103D60000E94DB0588EE93E00E94B50B80E00E9484
:103D7000DF08219683E0C83ED80709F0B7CFDF916E
:103D8000CF911F910F91FF90EF90DF90CF90BF9058
:103D9000AF9008952F923F924F925F926F927F92D1
:103DA0008F929F92AF92BF92CF92DF92EF92FF924B
:103DB0000F931F93DF93CF93CDB7DEB7C555D04098
:103DC0000FB6F894DEBF0FBECDBF5C0166967FAF25
:103DD0006EAF6697DE011196E4E9F0E080E10190B4
:103DE0000D928150E1F7CE0141960E94B732C50194
:103DF000880F991F880F991F64969FAF8EAF6497A5
:103E0000442455249DC080E00E94DF088824992422
:103E10007EC0F1018081B201680F711DCE01419613
:103E20000E947B328C539F4F61E370E00E94FE350D
:103E3000062F10E0C401B501A8010E94DB05C301F3
:103E4000B501A8010E94DB0577E0C72ED12CCA1866
:103E5000DB08C401B601A8010E94DB05C301B6015D
:103E6000A8010E94DB0567E0E62EF12CE01AF10ABA
:103E7000C401B501A7010E94DB05C301B501A7017B
:103E80000E94DB05C401B601A7010E94DB05C30146
:103E9000B601A7010E94DB05C401B801A5010E947B
:103EA000DB05C301B801A5010E94DB05C401B8010F
:103EB000A6010E94DB05C301B801A6010E94DB0533
:103EC000C401B701A5010E94DB05C301B701A5012B
:103ED0000E94DB05C401B701A6010E94DB05C301F6
:103EE000B701A6010E94DB050894A11CB11C84E067
:103EF00090E0280E391E94E0A916B10409F089CF8C
:103F00000894811C911CE4E08E16910479F051E034
:103F1000252E312C2C0E3D1E280C391CAA24BB2426
:103F200047E0642E712C6818790873CF66968EADC1
:103F30009FAD66970E94B50B84E090E0480E591E35
:103F40006496EEADFFAD64974E165F060CF45BCF42
:103F5000CB5ADF4F0FB6F894DEBF0FBECDBFCF9167
:103F6000DF911F910F91FF90EF90DF90CF90BF9066
:103F7000AF909F908F907F906F905F904F903F9009
:103F80002F9008952F923F924F925F926F927F925F
:103F90008F929F92AF92BF92CF92DF92EF92FF9259
:103FA0000F931F93DF93CF93CDB7DEB7C555D040A6
:103FB0000FB6F894DEBF0FBECDBF6C0166967FAF23
:103FC0006EAF6697DE011196E4EAF0E080E10190C1
:103FD0000D928150E1F7CE0141960E94B732C601A1
:103FE000880F991F880F991F64969FAF8EAF6497B3
:103FF00044245524A7E02A2E312C70C080E00E9472
:10400000DF08AA24BB2453C0F3018081B201680FEA
:10401000711DCE0141960E947B328C539F4F61E30C
:1040200070E00E94FE35062F10E0C501B601A80120
:104030000E94DB05C401B601A8010E94DB057101E5
:10404000EC18FD08C501B701A8010E94DB05C401F9
:10405000B701A8010E94DB05C101801B910B8C01F7
:10406000C501B601A8010E94DB05C401B601A80183
:104070000E94DB05C501B701A8010E94DB05C40150
:10408000B701A8010E94DB050894C11CD11CE4E023
:10409000F0E06E0E7F1EF4E0CF16D10409F0B4CF2D
:1040A0000894A11CB11C84E0A816B10469F0F1E0E9
:1040B0006F2E712C6C0E7D1E6A0C7B1CCC24DD24B3
:1040C00041018A189B08A0CF66968EAD9FAD66977A
:1040D0000E94B50BE4E0F0E04E0E5F1E64968EADDC
:1040E0009FAD6497481659060CF488CFCB5ADF4F22
:1040F0000FB6F894DEBF0FBECDBFCF91DF911F91F9
:104100000F91FF90EF90DF90CF90BF90AF909F9076
:104110008F907F906F905F904F903F902F90089579
:104120002F923F924F925F926F927F928F929F92C7
:10413000AF92BF92CF92DF92EF92FF920F931F93B5
:10414000DF93CF93CDB7DEB7C555D0400FB6F89407
:10415000DEBF0FBECDBF6C0166967FAF6EAF6697B8
:10416000DE011196E4EBF0E080E101900D928150C8
:10417000E1F7CE0141960E94B732C601880F991F20
:10418000880F991F64969FAF8EAF6497442455247F
:1041900007E0202E312C70C080E00E94DF08AA24A6
:1041A000BB2453C0F3018081B201680F711DCE01A1
:1041B00041960E947B328C539F4F61E370E00E94D6
:1041C000FE35062F10E0C501B801A6010E94DB05EF
:1041D000C401B801A6010E94DB057101EC18FD08BD
:1041E000C501B801A7010E94DB05C401B801A70100
:1041F0000E94DB05C101801B910B8C01C501B80138
:10420000A6010E94DB05C401B801A6010E94DB05DE
:10421000C501B801A7010E94DB05C401B801A701CF
:104220000E94DB050894C11CD11CE4E0F0E06E0E96
:104230007F1EF4E0CF16D10409F0B4CF0894A11C7E
:10424000B11C84E0A816B10469F011E0612E712C54
:104250006C0E7D1E6A0C7B1CCC24DD2441018A1867
:104260009B08A0CF66968EAD9FAD66970E94B50B5A
:10427000E4E0F0E04E0E5F1E64968EAD9FAD649755
:10428000481659060CF488CFCB5ADF4F0FB6F89476
:10429000DEBF0FBECDBFCF91DF911F910F91FF9079
:1042A000EF90DF90CF90BF90AF909F908F907F90D6
:1042B0006F905F904F903F902F9008952F923F9274
:1042C0004F925F926F927F928F929F92AF92BF9226
:1042D000CF92DF92FF920F931F93DF93CF93CDB7CF
:1042E000DEB7C355D0400FB6F894DEBF0FBECDBFCA
:1042F0006C0164967FAF6EAF6497DE011196E4ECBB
:10430000F0E080E101900D928150E1F7CE014196FD
:104310000E94B7321601220C331C220C331C662477
:1043200077245DC080E00E94DF08AA24BB243EC041
:10433000F4018081B301680F711DCE0141960E9486
:104340007B328C539F4F61E370E00E94FE35F62E66
:10435000C501B6014F2D50E00E94DB05C201B60138
:104360004F2D50E00E94DB0507E010E00C191D09FD
:10437000C501B8014F2D50E00E94DB05C201B80114
:104380004F2D50E00E94DB050894C11CD11C84E035
:1043900090E0880E991E94E0C916D10449F608945D
:1043A000A11CB11CE4E0AE16B10479F041E0842E0A
:1043B000912C8C0E9D1E8A0C9B1CCC24DD2437E096
:1043C000432E512C4A185B08B3CF64968EAD9FAD37
:1043D00064970E94B50B84E090E0680E791E621429
:1043E00073040CF49FCFCD5ADF4F0FB6F894DEBFA5
:1043F0000FBECDBFCF91DF911F910F91FF90DF9046
:10440000CF90BF90AF909F908F907F906F905F9074
:104410004F903F902F9008952F923F924F925F922E
:104420006F927F928F929F92AF92BF92CF92DF92C4
:10443000EF92FF920F931F93DF93CF9300D00F92D1
:10444000CDB7DEB7C82EB92E562E2DB73EB73B835B
:104450002A8387E0689FC0011124ADB7BEB7A81BAF
:10446000B90B0FB6F894BEBF0FBEADBF8DB69EB6EA
:104470000894811C911CDD242AC0ED2CFF248701A7
:10448000A3E0000F111FAA95E1F70E191F09080DEF
:10449000191DF801D08211820E9476368F70D801E2
:1044A00013968C931397C70181709070880F991F92
:1044B000880F991F14968C93B2E0EB22FF24EE0C28
:1044C000FF1CF801E5828D2D84708683D394D5146A
:1044D000A0F28C2D9B2D9C013901F2E0F983252C53
:1044E000332402C021E0298380E00E94DF086401B8
:1044F0004424AA24BB24A4C07401EA0CFB1CD701E9
:1045000011968C91882321F18D5F873009F486E024
:10451000F701E80FF11DD70112969C91915080810F
:10452000980F9083992319F0943009F06BC0F6012D
:104530008081D70111969C911197892780831196CC
:104540001C920E947636982F9F70F70193835AC071
:1045500087010D5F1F4FD70113968C911397882306
:1045600021F0815013968C934DC00E94763663E003
:1045700070E00E94FE35E1E0F0E002C0EE0FFF1FA8
:104580008A95E2F75E2FD6014C914E2730E018C095
:10459000832F90E0FC0173E0EE0FFF1F7A95E1F7A7
:1045A000E81BF90BE80DF91D2081421721F08181EC
:1045B0002827421721F425E0F801208350E03F5FCF
:1045C000351530F35523E1F0952F9D5F973009F4B1
:1045D00096E0F701E90FF11D8081882321F0D701D2
:1045E00012961C920DC022E0F701228339813130EE
:1045F00039F4953028F0D6018C91843008F450E0DD
:10460000F7015183D70114962C91149730E0159639
:104610000C91159710E01696EC91F0E0C901B801E5
:10462000AF012D5F3F4F0D5F1F4F33967F010E94FB
:1046300019094394E7E0F0E0CE0EDF1EAE0EBF1E78
:10464000451408F459CF80E293E00E94B50BF9813C
:10465000F23019F020E030E01BC0089461087108C6
:104660006114710409F43ECF3FCF822F90E0FC012A
:1046700063E0EE0FFF1F6A95E1F7E81BF90BE80D09
:10468000F91D808190E0821593050CF031E02F5FD9
:10469000251558F3332309F025CF8A819B810FB666
:1046A000F8949EBF0FBE8DBF0F900F900F90CF91CB
:1046B000DF911F910F91FF90EF90DF90CF90BF900F
:1046C000AF909F908F907F906F905F904F903F90B2
:1046D0002F9008952F923F924F925F926F927F9208
:1046E0008F929F92AF92BF92CF92DF92EF92FF9202
:1046F0000F931F93DF93CF9300D000D000D0CDB79E
:10470000DEB74C013A8329836230B0F4443030F490
:10471000433011F4EE2406C0EE2408C0453021F4E5
:10472000E2E0EE2E81E003C072E0E72E80E061302F
:1047300009F48260FF2462C0643038F5423058F4D6
:1047400080E0633009F481E0413009F48260EE24B6
:10475000FF24F39453C0862F90E0840F911D079798
:1047600051F4633021F0EE24E394FF2432C0EE24B0
:10477000E394FF2434C0633021F4EE24E394FF2457
:1047800036C0EE24E394FF2438C0842F90E0262F17
:1047900030E04230A0F4820F931F059741F464305B
:1047A00019F062E0E62E13C052E0E52E16C0653027
:1047B00019F442E0E42E19C032E0E32E1CC0820F4F
:1047C000931F079771F4643031F0EE24E394FF24D3
:1047D000F39481E013C0EE24E394FF24F39482E089
:1047E0000DC0653031F4EE24E394FF24F39483E0AC
:1047F00005C0EE24E394FF24F39480E004E010E08D
:1048000090E09C01227030703C832B8321E0222EAB
:10481000312C28223922FF2059F0C401B8010E940E
:104820007B32C82EC401B8010E949F32D82E0AC024
:10483000C401B8010E947B32D82EC401B8010E9485
:104840009F32C82E80E00E94DF08AA24B8E0BB2E69
:104850004D2C55246C2C77242A2D30E0249DC0014A
:10486000259D900D349D900D112468EA70E00E9402
:10487000FE35C62E8B819C81892B19F097E0961B03
:10488000C92E269DC001279D900D369D900D1124A7
:1048900068EA70E00E94FE35D62E2114310419F02A
:1048A000E7E0E61BDE2E1E821D82EE2029F48D81BC
:1048B0009E816D2D70E00EC0F1E0EF1639F48D2D64
:1048C00090E06C2D70E04D815E8106C08D2D90E0F2
:1048D0006D817E814C2D50E00E94DB052D813E8153
:1048E0002F5F3F4F3E832D8328303105F1F6A3948F
:1048F000BA9409F0B1CF89819A810E94B50B0C5FFF
:104900001F4F0432110509F086CF26960FB6F89492
:10491000DEBF0FBECDBFCF91DF911F910F91FF90F2
:10492000EF90DF90CF90BF90AF909F908F907F904F
:104930006F905F904F903F902F900895BF92CF92CD
:10494000DF92EF92FF920F931F93DF93CF93CDB738
:10495000DEB7C154D0400FB6F894DEBF0FBECDBF56
:10496000F82EE92E8E010F5F1F4FC8010E94B7324B
:104970002F2D3E2DC9016C01EE24B02E012F24C035
:104980000E94763666E070E00E94FE35F82E282FF1
:1049900030E08E2D90E08227932786709070892BCF
:1049A00039F4C901039666E070E00E94FE35F82EE6
:1049B0008B2D902F6E2D4F2D24EF31E00E946A2316
:1049C0000894C108D108EF2CC114D104C9F6CF5BFB
:1049D000DF4F0FB6F894DEBF0FBECDBFCF91DF9192
:1049E0001F910F91FF90EF90DF90CF90BF900895AF
:1049F0002F923F924F925F926F927F928F929F92EF
:104A0000AF92BF92CF92DF92EF92FF920F931F93DC
:104A1000DF93CF93CDB7DEB7C954D0400FB6F8942B
:104A2000DEBF0FBECDBF24969FAF8EAF24972696D4
:104A30007FAF6EAF26972E010894411C511CC20116
:104A40000E94B73266247724B1C08301159507957B
:104A5000C201B8010E947B327C01C201B8010E94F0
:104A60009F328C549F4F63E070E00E94FE358B01B3
:104A700080E00E94DF08C7018C549F4F63E070E024
:104A80000E94FE3588E0A82EB12CA61AB70AB8E01D
:104A90008B2E912C88E090E0801B910B2A969FAF83
:104AA0008EAF2A977501B7FE04C0EE24FF24EA18E2
:104AB000FB08EE9C1001EF9C300CFE9C300C112486
:104AC000C4016FE070E00E94FE3527966FAF279714
:104AD00028967FAF28972A960EAD1FAD2A97A8E09B
:104AE000CA2ED12CA80117FF04C044275527401B0C
:104AF000510BE114F10431F44115510519F460E052
:104B000070E018C09A012E0D3F1D35952795449FE2
:104B1000C001459F900D549F900D1124820D931D4F
:104B2000B9010E94FE35CB01820F931F63E070E054
:104B30000E94FE35660D771DC2010E947B329C01EA
:104B4000C6016FE070E00E94FE35FB01C9018C5484
:104B50009F4F64E370E00E94FE35AB0127968FAD56
:104B6000279728969FAD2897BF010E94DB058FE00D
:104B700090E0C80ED91E015F1F4F90E8C916D104FE
:104B800009F0B0CF8FE090E0880E991EA80EB91EF4
:104B900090E88916910409F085CF26968EAD9FADD9
:104BA00026970E94B50B0894611C711C24968EAD4B
:104BB0009FAD2497681679060CF447CFC75BDF4F8B
:104BC0000FB6F894DEBF0FBECDBFCF91DF911F911E
:104BD0000F91FF90EF90DF90CF90BF90AF909F909C
:104BE0008F907F906F905F904F903F902F9008959F
:104BF0002F923F924F925F926F927F928F929F92ED
:104C0000AF92BF92CF92DF92EF92FF920F931F93DA
:104C1000DF93CF93CDB7DEB76C970FB6F894DEBFB6
:104C20000FBECDBF9E8B8D8B788F6F8B2DB73EB710
:104C30003A8F298F80E00E94DF088F89988D880F36
:104C4000991FAF89B88D8A0F9B1F23E0880F991F8A
:104C50002A95E1F7EDB7FEB7E81BF90B0FB6F8940C
:104C6000FEBF0FBEEDBF8DB79EB701968B8F9C8F99
:104C70001C8A1B8AE2C10E94763664E070E00E94C2
:104C8000FE35AA2797FDA095BA2FBC01CD010E9441
:104C9000F4335B016C010E94763664E070E00E94A0
:104CA000FE35AA2797FDA095BA2FBC01CD010E9421
:104CB000F4337B018C010E94763662E070E00E9442
:104CC000FE35AA2797FDA095BA2FBC01CD010E9401
:104CD000F43320E030E040EA50E40E94EE326F838B
:104CE000788789879A87C601B50120E030E040E0E7
:104CF00050E40E94EE326B837C838D839E83C801D7
:104D0000B70120E030E040E050E40E94EE324B0179
:104D10005C0144245524CC24DD241CC06B817C819F
:104D20008D819E810E94C1337B018C01C501B4013C
:104D30000E94C1339B01AC01C701B901A2010E94CD
:104D4000DB050894411C511CC6010E94B50B80E094
:104D50000E94DF0824EF31E0C20ED31EB201882783
:104D600077FD8095982F0E94F4332F8138854985EF
:104D70005A850E94523387FDD1CF8B8D9C8D9C012B
:104D800029012224332486C08B819C81AD81BE8180
:104D9000F20180839183A283B383D20114968D9212
:104DA0009D92AD92BC9217978F819885A985BA85FF
:104DB00080879187A287B3870E9476368C010E94F4
:104DC00076367C010E9476366C01C80168EC70E092
:104DD0000E94FE35AA2797FDA095BA2FBC01CD01F0
:104DE0000E94F43320E030E048EC52EC0E9459334A
:104DF00020E030E040E85FE30E94EE32D2011C96F2
:104E00006D937D938D939C931F97C70168EC70E021
:104E10000E94FE35AA2797FDA095BA2FBC01CD01AF
:104E20000E94F43320E030E048EC52EC0E94593309
:104E300020E030E040E85FE30E94EE32F201608B58
:104E4000718B828B938BC60168EC70E00E94FE35FB
:104E5000AA2797FDA095BA2FBC01CD010E94F4337B
:104E600020E030E048EC52EC0E94593320E030E082
:104E700040E85FE30E94EE32D20154966D937D9339
:104E80008D939C9357970894211C311CE8E1F0E026
:104E90004E0E5F1E2F89388D221633060CF474CF08
:104EA0001A821982A981BA81BD01882777FD809570
:104EB000982F0E94F4332DEC3CEC4CEC5DE30E9407
:104EC000EE3220E030E040EA51E40E9459330E9483
:104ED0008C357B018C0120E030E040E251E40E94FF
:104EE000E13420E030E040E85FE30E94EE326F877B
:104EF000788B898B9A8BC801B70120E030E040E0C5
:104F00005FE30E94E1346B877C878D879E872B8DC2
:104F10003C8DC9012C012224332475C0F201648523
:104F20007585868597852F85388949895A890E9494
:104F300059339B01AC01D2016D917D918D919C9172
:104F40000E94EE323B014C01F20160837183828347
:104F5000938360897189828993892F8538894989EA
:104F60005A890E9459339B01AC01D20114966D916C
:104F70007D918D919C9117970E94EE327B018C015F
:104F8000F201648375838683978364897589868932
:104F900097892F85388949895A890E945933D201C6
:104FA00018962D913D914D915C911B970E94EE3288
:104FB0002B853C854D855E850E94ED325B016C0141
:104FC000F2016087718782879387C401B3010E94D1
:104FD000C1333B014C01C801B7010E94C1337B01C1
:104FE0008C01C601B5010E94C1339B01AC01C30114
:104FF000B701A9010E94DB050894211C311C28E19E
:1050000030E0420E531E8F89988D281639060CF415
:1050100085CF88EE93E00E94B50B80E00E94DF0808
:10502000A981BA811196BA83A983599709F03ACF19
:10503000EB89FC893196FC8BEB8B2B893C898D8924
:105040009E89281739070CF416CEA98DBA8D0FB694
:10505000F894BEBF0FBEADBF6C960FB6F894DEBF1E
:105060000FBECDBFCF91DF911F910F91FF90EF90B9
:10507000DF90CF90BF90AF909F908F907F906F9078
:105080005F904F903F902F9008954F925F926F9254
:105090007F928F929F92AF92BF92CF92DF92EF92C8
:1050A000FF920F931F93CF93DF933C014B01AA24F0
:1050B000BB2447E0442E512C36C0C0E0D0E0620152
:1050C000CC1ADD0A80E090E060E070E0AE0127E0FD
:1050D00030E000E010E076010E94B80A80E090E045
:1050E000BE0140E050E027E030E08601EE24FF24DE
:1050F0000E94B80AC4010E94B50B89E761E070E024
:105100000E94C40B8AE76FEF7FEF0E94C40B88E711
:105110006FEF7FEF0E94C40B2196C830D10579F65E
:105120000894A11CB11CA614B7043CF2DF91CF91E6
:105130001F910F91FF90EF90DF90CF90BF90AF90B5
:105140009F908F907F906F905F904F9008952F92D7
:105150003F924F925F926F927F928F929F92AF9207
:10516000BF92CF92DF92EF92FF920F931F93DF9344
:10517000CF93CDB7DEB739014A01A60195010E9450
:10518000ED325B016C01C401B3012D893E894F8969
:10519000588D0E94ED323B014C01C801B701298DA9
:1051A0003A8D4B8D5C8D0E94ED321B012C01C601A6
:1051B000B501A60195010E94E1347B018C01C40177
:1051C000B301A40193010E94E1349B01AC01C80129
:1051D000B7010E94EE327B018C01C201B101A20134
:1051E00091010E94E1349B01AC01C801B7010E940A
:1051F000EE320E944E35CF91DF911F910F91FF90BB
:10520000EF90DF90CF90BF90AF909F908F907F9066
:105210006F905F904F903F902F9008952F923F9204
:105220004F925F926F927F928F929F92AF92BF92B6
:10523000CF92DF92EF92FF920F931F93DF93CF9362
:10524000CDB7DEB7A0970FB6F894DEBF0FBECDBFC7
:105250009A87898780E00E94DF081A82198216C126
:1052600029813A81B901882777FD8095982F0E947E
:10527000F4335B016C0120E030E048E452E40E942A
:1052800059337B018C01C8010E94443520E030E095
:1052900040E250E40E94E13420E030E040E650E497
:1052A0000E94EE326B8B7C8B8D8B9E8BB701C8017D
:1052B0000E94563320E030E040E250E40E94E134A6
:1052C00020E030E040E650E40E94EE326F87788BB9
:1052D000898B9A8BC601B50120E030E040EF51E4A4
:1052E0000E9459330E9456339B01AC010E94EE325A
:1052F00020E030E040E650E40E94EE326B877C878D
:105300008D879E87C601B50120E030E046E153E479
:105310000E9459330E94443520E030E040E050E4E0
:105320000E94EE326D837E838F83988780E00E9497
:10533000DF081C821B8298C08DB79EB708970FB6F6
:10534000F8949EBF0FBE8DBF4DB65EB60894411C4B
:10535000511C6B8D7C8D8D8D9E8D0E94F4333B0195
:105360004C016F89788D898D9A8D0E94F4335B0191
:105370006C01AF8DB8A1BD01882777FD8095982F6E
:105380000E94F4337B018C012F85388949895A8921
:10539000C901DA01F20180839183A283B3832B8553
:1053A0003C854D855E85C901DA0184839583A6839A
:1053B000B783C401B301A6019501EB89FC896D880F
:1053C0004E885F01C62CD42C0E94A7287B018C013B
:1053D0002DB73EB7285F3F4F0FB6F8943EBF0FBEC4
:1053E0002DBF2D813E814F8158850E94DD341816D6
:1053F000CCF46D817E818F81988520E030E040E89B
:105400005FE30E94EE329B01AC01C801B7010E942C
:10541000523388233CF48B819C81B1014F8D58A17C
:105420000E94DB058F8D98A1019698A38F8F089716
:1054300009F082CF0894211C311C98E02916310410
:1054400061F018A21F8EC101AA2797FDA095BA2F5F
:105450008F8B988FA98FBA8F6FCFAB81BC8111963C
:10546000BC83AB83189769F0222433248B819C8101
:10547000AA2797FDA095BA2F8B8F9C8FAD8FBE8FDB
:10548000E0CFA981BA811196BA83A983E981FA8113
:1054900029853A85E217F3070CF4E2CEA0960FB601
:1054A000F894DEBF0FBECDBFCF91DF911F910F915A
:1054B000FF90EF90DF90CF90BF90AF909F908F9034
:1054C0007F906F905F904F903F902F9008956F92D4
:1054D0007F928F929F92AF92BF92CF92DF92EF9284
:1054E000FF920F931F9339014A01A80197010E946F
:1054F000ED327B018C01C401B301A60195010E942C
:10550000ED325B016C01C801B701A80197010E944F
:10551000E1347B018C01C601B501A60195010E9411
:10552000E1349B01AC01C801B7010E94EE320E9438
:105530004E351F910F91FF90EF90DF90CF90BF906D
:10554000AF909F908F907F906F9008952F923F9291
:105550004F925F926F927F928F929F92AF92BF9283
:10556000CF92DF92EF92FF920F931F93DF93CF932F
:10557000CDB7DEB728970FB6F894DEBF0FBECDBF0C
:105580009A8389836624772480C080E00E94DF08A4
:1055900088249924C301AA2797FDA095BA2F8B834D
:1055A0009C83AD83BE8366C0C201B1010E94F43307
:1055B0007B018C01AF81B885BD01882777FD80957F
:1055C000982F0E94F4335B016C0160E070E080E68C
:1055D00090E49B01AC010E94672A25E534E64EE188
:1055E00051E40E94593320E030E040E051E40E9451
:1055F000E13426E636E646EA5FE30E9459337B0152
:105600008C016B817C818D819E810E94F43320E02E
:1056100030E048E452E40E9459339B01AC01C801D8
:10562000B7010E94EE320E94443520E030E040E8AD
:1056300050E40E94E13420E030E040E850E40E9471
:10564000EE320E94C1339B01AC01C4016F817885A9
:10565000A9010E94DB05EF81F8853196F887EF8379
:10566000389709F0A1CF0894811C911CF8E08F169F
:10567000910441F018861F821401442437FC4094A1
:10568000542C92CF0894611C711C29813A816216B6
:1056900073060CF47ACF28960FB6F894DEBF0FBECF
:1056A000CDBFCF91DF911F910F91FF90EF90DF90D1
:1056B000CF90BF90AF909F908F907F906F905F90B2
:1056C0004F903F902F9008952F923F924F925F926C
:1056D0006F927F928F929F92AF92BF92CF92DF9202
:1056E000EF92FF920F931F93DF93CF93CDB7DEB767
:1056F0002C970FB6F894DEBF0FBECDBF9A8789876F
:10570000662477244EC02B853C85B901882777FD18
:105710008095982F0E94F4332D813E814F815885CA
:105720000E9459339B01AC01C201B1010E94EE32CB
:105730000E94443529813A814B815C810E94E13489
:1057400020E030E040E850E40E94EE327B018C0122
:105750000E94C1334B015C0160E070E080EE90E498
:10576000A80197010E94ED320E94C1336B017C01B8
:105770008DEF9FEF6B857C85A4012AE030E08B01E3
:1057800076010E9401068B859C8501969C878B87FC
:10579000089709F0B8CF80E00E94DF080894611CE8
:1057A000711CE985FA856E167F060CF04EC0B301B8
:1057B000882777FD8095982F0E94F4337B018C0118
:1057C00020E030E048EC52E40E9459330E94443516
:1057D00020E030E040E050E40E94EE3220E030E093
:1057E00040E85FE30E94EE326D837E838F8398876B
:1057F000C801B70120E030E048E453E40E94593387
:105800000E94443520E030E040E85FE30E94EE3241
:1058100020E030E040EC50E40E94E13420E030E051
:1058200040E450E40E94EE3269837A838B839C8348
:10583000C801B70120E030E040E252E40E94593351
:105840001B012C011C861B865ECF2C960FB6F8948C
:10585000DEBF0FBECDBFCF91DF911F910F91FF90A3
:10586000EF90DF90CF90BF90AF909F908F907F9000
:105870006F905F904F903F902F9008952F923F929E
:105880004F925F926F927F928F929F92AF92BF9250
:10589000CF92DF92EF92FF920F931F93DF93CF93FC
:1058A000CDB7DEB76A970FB6F894DEBF0FBECDBF97
:1058B000988B8F871A821982AAC0298D3A8DB901D7
:1058C000882777FD8095982F0E94F4335B016C0147
:1058D0002F81388549855A850E9459339B01AC0137
:1058E0006B857C858D859E850E94EE327B018C01C7
:1058F0000E9444353B014C01C801B7010E94563358
:105900001B012C01C801B70123EC35EF48E450E43A
:105910000E94EE327B018C01C8010E9444356B83EA
:105920007C838D839E83B701C8010E9456337B011F
:105930008C01C601B5010E94C133698B7A8B8B8BB8
:105940009C8BC401B30120E030E040EA50E40E94A7
:10595000E13420E030E040E850E40E94EE320E9462
:10596000C1336D8B7E8B8F8B988FC201B10120E08C
:1059700030E040EA50E40E94E13420E030E040E8CA
:1059800050E40E94EE320E94C1332B013C016B8136
:105990007C818D819E8120E030E040E251E40E94D4
:1059A000E13420E030E040E850E40E94EE320E9412
:1059B000C1334B015C01C801B70120E030E040E297
:1059C00051E40E94E13420E030E040E850E40E94DD
:1059D000EE320E94C1336B017C0189899A896D89FD
:1059E0007E89A2019C01840176010E940106898DB5
:1059F0009A8D01969A8F898F089709F05ECF80E083
:105A00000E94DF08E981FA813196FA83E9832981CE
:105A10003A818F8598892817390784F5B901882735
:105A200077FD8095982F0E94F4337B018C0120E054
:105A300030E048E452E40E9459336B877C878D87BD
:105A40009E87C801B70120E030E048E453E40E949B
:105A500059330E94443520E030E040EE50E40E948B
:105A6000E13420E030E040E251E40E94EE326F8306
:105A7000788789879A871A8E198E1FCF6A960FB6F4
:105A8000F894DEBF0FBECDBFCF91DF911F910F9174
:105A9000FF90EF90DF90CF90BF90AF909F908F904E
:105AA0007F906F905F904F903F902F90089581303E
:105AB00019F48CE190E002C080E090E0DC01A35298
:105AC000BF4F20E030E009C0FD018491FB01E20FEF
:105AD000F31F80832F5F3F4F119624173507A4F3E0
:105AE00008951F93142F90E023E0880F991F2A95A3
:105AF000E1F7860F911D89539E4F0E94863690E0F4
:105B000002C0959587951A95E2F781701F910895C7
:105B1000EF92FF920F931F93CF93DF937B01C82FD8
:105B2000D0E033E0CC0FDD1F3A95E1F7C953DE4FEB
:105B300000E010E0CE010E948636F701E00FF11F71
:105B400080830F5F1F4F21960830110599F7DF9171
:105B5000CF911F910F91FF90EF900895EF92FF92D8
:105B60000F931F93CF93DF937B01805295E0899F22
:105B70008001112400501040C0E0D0E0C8010E9414
:105B80008636F701EC0FFD1F808321960F5F1F4FB4
:105B9000C530D10599F7DF91CF911F910F91FF90FB
:105BA000EF900895AF92BF92DF92EF92FF920F9322
:105BB0001F93CF93DF93182F092F80E00E94DF08F7
:105BC00082B3837E82BBE12FF02FE432F10508F02F
:105BD0008FC3E65DFF4FEE0FFF1F0590F491E02DA0
:105BE000099416E083E090E068EE73E0412F0E9494
:105BF000F0101F5F1D30B1F70E946C1784E690E033
:105C00000E94AB1880E00E94DF0802EC11E080E403
:105C100090E0B8010E945E210E5110400E31110536
:105C2000B1F76AC38CED95E06AE070E00E943E2C0B
:105C300080EA9FE06AE070E00E94642B80E00E94AE
:105C4000DF0880EB94E06CE043E050E00E94040F3A
:105C500084E893E06CE043E050E00E94040F88E5A4
:105C600092E06CE043E050E00E94040F8CE291E08F
:105C70006CE043E050E00E94040F84E690E06CE0AA
:105C800043E050E00E94040F8AE090E06CE043E0C3
:105C900050E00E94040F8CE291E064EF71E00E94FA
:105CA000FA1988EC90E064E873E00E948D198CE2A8
:105CB00091E064EF71E00E94902088E592E06CE250
:105CC00071E01FC28CEB92E066E044E050E0C9C195
:105CD00084E190E06CED70E040ED57E00E94F41636
:105CE0000BC385E090E061E070E00E948A1685E0D9
:105CF00090E060E070E00E948A1685E090E061E04C
:105D000070E00E948A1685E090E060E070E00E94FA
:105D10008A16F2C284E190E068EE73E00E94D41526
:105D2000EBC282E090E0C4C188E592E060E971E0F6
:105D30000E94C21F00E010E0B80163707070A801FB
:105D40004470507081E090E022EC31E00E94921D9E
:105D50000F5F1F4F0830110579F780E293E060E094
:105D600070E00E94511D80E293E061E070E00E94CB
:105D7000511D80E293E060E070E00E94511D80E2DE
:105D800093E061E070E00E94511DB6C28AE790E0A6
:105D900068E572E00E941B1E88E790E068E572E00B
:105DA0000E941B1E89E790E068E572E00E941B1EBE
:105DB0008AE790E068E572E00E941B1E88E790E0A9
:105DC00068E572E00E941B1E89E790E068E572E0DA
:105DD0000E941B1E8AE790E068E572E00E94411E67
:105DE00088E790E068E572E00E94411E89E790E054
:105DF00068E572E00E94411E8AE790E068E572E083
:105E00000E94411E88E790E068E572E00E94411E12
:105E100089E790E068E572E00E94411E80E00E9400
:105E2000DF086AC280E00E94DF0880E090E060E264
:105E300073E04FEF50E00E943E0E80E090E060E2A1
:105E400073E040E050E00E943E0E81E090E060E2AE
:105E500073E04FEF50E00E943E0E81E090E060E280
:105E600073E040E050E00E943E0E46C28AE766E2E0
:105E700072E048E853E120E030E00E9400158AE734
:105E800066E272E048E853E121E030E00E9400154C
:105E90008AE766E272E048E853E120E030E00E94E1
:105EA00000158AE766E272E048E853E121E030E05D
:105EB0000E94001588E766E272E048E853E120E0BE
:105EC00030E00E94001588E766E272E048E853E19E
:105ED00021E030E00E94001589E766E272E048E8C0
:105EE00053E120E030E00E94001589E766E272E0AD
:105EF00048E853E121E030E00E940015FDC18CEB41
:105F000092E00E948513F8C181E090E06AE770E0BA
:105F100041E050E024E630E008EE13E00E94CD17A7
:105F2000EBC184ED90E0E6C180E00E94DF08C0E0B4
:105F3000D0E00E9476368C010E9476367C010E9469
:105F40007636FC01C80164E070E00E94FE358C01E9
:105F5000C70164E070E00E94FE359C01CF0164E05F
:105F600070E00E94FE35AC01C801B9010E94DB055A
:105F70002196C431D105E9F682E390E068E572E04C
:105F8000B4C18AE760E070E048EC50E021E030E026
:105F90000E9446148CED95E00E94B50B8AE761E003
:105FA00070E048EC50E021E030E00E9446148CEDB7
:105FB00095E00E94B50B8AE760E070E048EC50E0A5
:105FC00022E030E00E9446148CED95E00E94B50B73
:105FD0008AE761E070E048EC50E022E030E00E94A7
:105FE00046148CED95E00E94B50B89E760E070E007
:105FF00048EC50E021E030E00E9446148CED95E042
:106000000E94B50B89E761E070E048EC50E021E0C8
:1060100030E00E9446148CED95E00E94B50B6CC1F7
:106020008AEF90E068E572E041E022E04CC084E055
:1060300090E068EE73E010E0412F0E94F01084E0E1
:1060400090E068EE73E0412F14C088EC90E064EFBC
:1060500071E00E943A1050C18CEB92E062E043E0A4
:1060600050E00E94040F48C182E090E068EE73E0C7
:1060700041E00E94F01040C188EE93E061E071E0E1
:106080000E94980F39C188EC90E064EF71E00E94A3
:10609000871032C10E946C172FC182E090E068EE39
:1060A00073E042E0E6CF0E946A1326C181E090E0EF
:1060B0006AE770E04FEF5FEF2DCF8AEF90E068E581
:1060C00072E041E023E00E94491A16C184E690E0A4
:1060D0000E949E2411C188E592E06CE271E00E946A
:1060E0005E2188E592E06CE271E00E94C21F88E5C3
:1060F00092E06CE271E00E94902084E690E060ED16
:1061000077E00E94CA1EF8C080E293E069E170E087
:106110000E94F824F1C084E690E063E00E940C2223
:10612000EBC08AE090E068E270E00E94F825E4C0ED
:1061300080E00E94DF08C0E0D0E00E9476368C014B
:106140000E9476367C010E947636FC01C80164E02C
:1061500070E00E94FE358C010E5F1F4FC70164E0A6
:1061600070E00E94FE359C012E5F3F4FCF0164E03E
:1061700070E00E94FE35AC014E5F5F4FC801B9016F
:106180000E94DB052196CA30D105B9F688EC90E073
:106190006CEB72E00E944E3280E00E94DF08C0E0AB
:1061A000D0E00E9476368C010E9476367C010E94F7
:1061B0007636FC01C80164E070E00E94FE358C0177
:1061C0000E5F1F4FC70164E070E00E94FE359C0126
:1061D0002E5F3F4FCF0164E070E00E94FE35AC01BE
:1061E0004E5F5F4FC801B9010E94DB052196CF3099
:1061F000D105B9F68CED90E06CEB72E00E944E3266
:1062000080E00E94DF08C0E0D0E00E9476368C017A
:106210000E9476367C010E947636FC01C80164E05B
:1062200070E00E94FE358C010E5F1F4FC70164E0D5
:1062300070E00E94FE359C012E5F3F4FCF0164E06D
:1062400070E00E94FE35AC014E5F5F4FC801B9019E
:106250000E94DB052196C231D105B9F68CE291E0AE
:1062600068E572E00E944E3280E00E94DF08C0E0E4
:10627000D0E057E0A52EB12C0E9476368C010E940A
:1062800076367C010E9476369C01C80164E070E09D
:106290000E94FE3542E0D42ED80EC70166E070E0C1
:1062A0000E94FE35082F0F5F10E0C90164E070E026
:1062B0000E94FE3592E0F92EF80E8D2D90E0B80187
:1062C0004F2D50E00E94DB05B501601B710B8D2D39
:1062D00090E04F2D50E00E94DB052196C830D1059B
:1062E00059F68CE291E06CEB72E00E944E3204C0F1
:1062F0008CE291E00E94FA18DF91CF911F910F91EB
:10630000FF90EF90DF90BF90AF90089540E050E095
:1063100018C0FB01E20FF31FDF01A35CBE4F9C918D
:10632000E358FE4F80819817A9F42F5F3F4F283024
:10633000310579F74F5F5F4F4830510511F480E028
:10634000089520E030E0BA0183E0660F771F8A9558
:10635000E1F7DFCF81E008955F926F927F928F9295
:106360009F92AF92BF92CF92DF92EF92FF920F93E4
:106370001F93CF93DF9380E00E94FC08C0E0D0E041
:1063800021E0822E912C74010C2E02C0EE0CFF1C19
:106390000A94E2F7BE2CA0E0B0E05C2E5A9492E0A2
:1063A000692E6C0E5EC0812F992787FD909583FD25
:1063B00028C0940102C0220F331F8A95E2F7922F62
:1063C000372D632F772767FD709563FD17C02C2D40
:1063D000E22FFF27E7FDF095E3FD0DC083E0EE0F10
:1063E000FF1F8A95E1F7E60FF71FE358FE4F808104
:1063F000892309F00F5F2F5F2D1551F73F5F3A1585
:1064000001F71F5F161579F69A0163E0220F331F1B
:106410006A95E1F72A0F3B1FF901E358FE4F80818F
:1064200090E08E219F21892B19F0053049F402C09C
:10643000043031F4F901E35CFE4F80818B298083C5
:106440004F5F5F4F4830510541F0152D00E0C42EDD
:10645000CA9422E0D22ED40EA6CF1196A830B10550
:1064600041F040E050E07A2E7A9492E0A92EAA0EF4
:10647000ECCF2196C830D10509F085CFDF91CF91BF
:106480001F910F91FF90EF90DF90CF90BF90AF9052
:106490009F908F907F906F905F900895DF92EF9222
:1064A000FF920F931F93CF93DF937C018B01C0E08A
:1064B000D0E038E0D32E14C082B38D2582BB0E9479
:1064C000AC31CE0187709070892B21F40E94863107
:1064D000882349F00E948A0DC8010E94B50B2196BD
:1064E000CE15DF054CF3DF91CF911F910F91FF90F7
:1064F000EF90DF900895AC0177FD02C020E004C06A
:10650000709561957F4F21E06F77707061347105F0
:106510002CF06054704081E0821B282FFA01E60FB6
:10652000F71F222339F0808190E066277727681BC8
:10653000790B03C08081682F70E0CB010895605E05
:106540007F4F6F777070FC01E60FF71F61347105A4
:106550004CF0E054F040808190E022273327281B44
:10656000390B03C08081282F30E0C9010895EF92D4
:10657000FF920F931F93CF93DF937C01C0E0D0E095
:10658000BE01882777FD8095982F0E94F4332BED6C
:106590003FE049E450E40E94E13420E030E040E88C
:1065A0005CE30E94E1340E94443587010C0F1D1FFB
:1065B00020E030E045E353E40E94E1340E94C6331A
:1065C000F80160832196C134D105D1F6DF91CF91D6
:1065D0001F910F91FF90EF9008955058BB27AA2765
:1065E0000ED0A0C169D130F06ED120F031F49F3FC0
:1065F00011F41EF45EC10EF4E095E7FB54C1E92FDF
:10660000B3D180F3BA17620773078407950718F0B0
:1066100071F49EF5CBC10EF4E0950B2EBA2FA02D90
:106620000B01B90190010C01CA01A0011124FF273F
:10663000591B99F0593F50F4503E68F11A16F0403A
:10664000A22F232F342F4427585FF3CF4695379539
:106650002795A795F0405395C9F77EF41F16BA0BFE
:10666000620B730B840BBAF09150A1F0FF0FBB1FAC
:10667000661F771F881FC2F70EC0BA0F621F731FF5
:10668000841F48F4879577956795B795F7959E3F52
:1066900008F0B3CF9395880F08F09927EE0F9795E0
:1066A00087950895DCD008F481E0089514D1E3952E
:1066B0004AC10CD037C107D140F0FED030F021F4F0
:1066C0005F3F19F0F0C0511172C1F3C04DD198F382
:1066D0009923C9F35523B1F3951B550BBB27AA2763
:1066E00062177307840738F09F5F5F4F220F331FD5
:1066F000441FAA1FA9F333D00E2E3AF0E0E830D0A1
:1067000091505040E695001CCAF729D0FE2F27D0A3
:10671000660F771F881FBB1F261737074807AB0771
:10672000B0E809F0BB0B802DBF01FF2793585F4FE6
:106730002AF09E3F510568F0B6C039C15F3FECF3C7
:10674000983EDCF3869577956795B795F7959F5FAB
:10675000C9F7880F911D9695879597F90895E1E0FF
:10676000660F771F881FBB1F621773078407BA075E
:1067700020F0621B730B840BBA0BEE1F88F7E095B9
:10678000089504D06894B11112C10895F5D088F02D
:106790009F5790F0B92F9927B751A0F0D1F0660F0D
:1067A000771F881F991F1AF0BA95C9F712C0B13028
:1067B00081F0FCD0B1E00895F9C0672F782F8827C9
:1067C000B85F39F0B93FCCF3869577956795B39567
:1067D000D9F73EF490958095709561957F4F8F4FD6
:1067E0009F4F0895E89409C097FB3EF490958095DB
:1067F000709561957F4F8F4F9F4F9923A9F0F92F87
:1068000096E9BB279395F695879577956795B79504
:10681000F111F8CFFAF4BB0F11F460FF1BC06F5FEA
:106820007F4F8F4F9F4F16C0882311F096E911C0FC
:10683000772321F09EE8872F762F05C0662371F01D
:1068400096E8862F70E060E02AF09A95660F771F31
:10685000881FDAF7880F9695879597F90895990F0D
:106860000008550FAA0BE0E8FEEF16161706E8071A
:10687000F907C0F012161306E407F50798F0621B3B
:10688000730B840B950B39F40A2661F0232B242B10
:10689000252B21F408950A2609F4A140A6958FEF2F
:1068A000811D811D089597F99F6780E870E060E081
:1068B00008959FEF80EC089500240A941616170699
:1068C00018060906089500240A94121613061406E1
:1068D00005060895EECF50D0E8F3E894E0E0BB273A
:1068E0009F57F0F02AED3FE049EC06C0EE0FBB0FDA
:1068F000661F771F881F28F0B23A62077307840764
:1069000028F0B25A620B730B840BE3959A9572F7D9
:10691000803830F49A95BB0F661F771F881FD2F717
:1069200090481CC1092E0394000C11F4882352F0E6
:10693000BB0F40F4BF2B11F460FF04C06F5F7F4FAB
:106940008F4F9F4F0895EF93E0FF06C0A2EA2AED14
:106950003FE049EC5FEB53DEE5DF0F90039401FC71
:106960009058ECE9F0E00DC157FD9058440F551FC9
:1069700059F05F3F71F04795880F97FB991F61F0C1
:106980009F3F79F087950895121613061406551F38
:10699000F2CF4695F1DF08C0161617061806991FA4
:1069A000F1CF86957105610508940895E894BB2799
:1069B00066277727CB0197F9089551DF08F48FEF09
:1069C00008950BD0AFCF78DF28F07DDF18F0952346
:1069D00009F069CF6ECF1124EACFC6DFA0F3959FEF
:1069E000D1F3950F50E0551F629FF001729FBB27B6
:1069F000F00DB11D639FAA27F00DB11DAA1F649F62
:106A00006627B00DA11D661F829F2227B00DA11D14
:106A1000621F739FB00DA11D621F839FA00D611D9A
:106A2000221F749F3327A00D611D231F849F600DBB
:106A3000211D822F762F6A2F11249F5750408AF0F4
:106A4000E1F088234AF0EE0FFF1FBB1F661F771F80
:106A5000881F91505040A9F79E3F510570F023CFF9
:106A6000A6CF5F3FECF3983EDCF38695779567956C
:106A7000B795F795E7959F5FC1F7FE2B880F911D9E
:106A80009695879597F908959F9325DF0F9007FCBA
:106A9000EE5F59CF11F40EF40CCF5EC06DDFD0F372
:106AA0009923D9F3CEF39F57550B87FF63D000246A
:106AB000A0E640EA900180585695979528F4805CAE
:106AC000660F771F881F20F026173707480730F416
:106AD000621B730B840B202931294A2BA69517942E
:106AE0000794202531254A2758F7660F771F881FFE
:106AF00020F026173707480730F4620B730B840B1E
:106B0000200D311D411DA09581F7B901842F9158A9
:106B1000880F969587950895DF93D92FDCDEE6954B
:106B2000D7952AED3FE049E45FE3B33A6207730784
:106B300084079507D7952AF0A2EA49EC90685FDDB3
:106B4000F1DEEAEBF0E01DD0DD0F0BF02BD0DD0F16
:106B50000BF49058DF9108959F3F31F0915020F44D
:106B6000879577956795B795880F911D9695879529
:106B700097F9089591505040660F771F881FD2F7FC
:106B800008959F938F937F936F93FF93EF939B0150
:106B9000AC0117DFEF91FF910CD02F913F914F91F6
:106BA0005F910FCF9B01AC0160E070E080E89FE354
:106BB00080CDDF93CF931F930F93FF92EF92DF92DD
:106BC0007B018C01689405C0DA2EEF0106DFFE011F
:106BD000E894A5912591359145915591AEF3EF013A
:106BE0000EDDFE019701A801DA9479F7DF90EF90AE
:106BF000FF900F911F91CF91DF91089597FB092E80
:106C000007260AD077FD04D00CD006D000201AF455
:106C1000709561957F4F0895F6F7909581959F4FF8
:106C20000895AA1BBB1B51E107C0AA1FBB1FA617D3
:106C3000B70710F0A61BB70B881F991F5A95A9F725
:106C400080959095BC01CD010895A0E0B0E0EBE205
:106C5000F6E30C94D036EC01A880B980CA80DB80C2
:106C6000A114B104C104D10441F484E2A82E89ED39
:106C7000B82E8BE5C82E87E0D82EC601B5012DE1D0
:106C800033EF41E050E00E94AD3627EA31E440E0C6
:106C900050E00E948E367B018C01C601B5012DE1CA
:106CA00033EF41E050E00E94AD36CA01B9012CEE4D
:106CB00034EF4FEF5FEF0E948E366E0D7F1D801F09
:106CC000911F97FF04C061507040804090486883D6
:106CD00079838A839B839B013F77C901CDB7DEB758
:106CE000EAE00C94EC360E942536089581E391E0A9
:106CF0000E9425360895A0E0B0E080933101909382
:106D00003201A0933301B09334010895E199FECF8D
:106D10009FBB8EBBE09A99278DB30895629FD001E7
:106D2000739FF001829FE00DF11D649FE00DF11D46
:106D3000929FF00D839FF00D749FF00D659FF00DF5
:106D40009927729FB00DE11DF91F639FB00DE11DE2
:106D5000F91FBD01CF011124089597FB092E0526C7
:106D60000ED057FD04D04BD00AD0001C38F45095FB
:106D70004095309521953F4F4F4F5F4F0895F6F75F
:106D800090958095709561957F4F8F4F9F4F089597
:106D90002F923F924F925F926F927F928F929F922B
:106DA000AF92BF92CF92DF92EF92FF920F931F9319
:106DB000CF93DF93CDB7DEB7CA1BDB0B0FB6F894CA
:106DC000DEBF0FBECDBF09942A88398848885F840A
:106DD0006E847D848C849B84AA84B984C884DF807B
:106DE000EE80FD800C811B81AA81B981CE0FD11D5F
:106DF0000FB6F894DEBF0FBECDBFED010895A1E23E
:106E00001A2EAA1BBB1BFD010DC0AA1FBB1FEE1F24
:106E1000FF1FA217B307E407F50720F0A21BB30B6F
:106E2000E40BF50B661F771F881F991F1A9469F7EB
:106E300060957095809590959B01AC01BD01CF0147
:066E40000895F894FFCF55
:106E46004D555349430031003200330034003500BC
:106E5600F401010000010203040506070101020313
:106E660004050606020203030404050503030303DF
:106E760004040404312B26232B231D1A261D15106A
:106E860023191007312B26232B231D1A261D151017
:106E960023191007312B26232B231D1A261D151007
:106EA60023191007312B26232B231D1A261D1510F7
:106EB600231910075355504552544543482D4954FC
:106EC60020444F5420434F4D2020202053555045F9
:106ED60052544543482D495420444F5420434F4D66
:106EE600005355504552544543482D495420444F6C
:106EF6005420434F4D202053555045525445434846
:106F06002D495420444F5420434F4D004641494C8F
:066F160000010000000074
:00000001FF
